:020000040000FA
:040200006BEF03F0AD
:040208000EEF01F004
:080218002DEF01F0D8CF01F039
:10022000E0CF02F0006EF3CF03F0F4CF04F0F0ACB7
:100230001DEF01F0F0B066EC0BF0A2A023EF01F08F
:10024000A1B018EC09F003C0F3FF04C0F4FF0050A4
:1002500002C0E0FF01C0D8FF1000D8CF06F0E8CF01
:1002600005F0E0CF07F0F3CF08F0F4CF09F0F0BCD1
:100270003DEF01F0F0B066EC0BF0A2B043EF01F0FF
:10028000A1B018EC09F0A2B04CEF01F0AECFE8FF3E
:100290006ECFE8FF52EF01F09EBAFCEC0EF0A4BA6C
:1002A00067EC0FF008C0F3FF09C0F4FF07C0E0FFE0
:0A02B00005C0E8FF06C0D8FF1000EB
:10030000F95000011150F926D4EF29F0D6EF29F069
:10031000E3EF29F0F8EF29F006EF2AF014EF2AF0C6
:1003200022EF2AF030EF2AF040EF2AF04EEF2AF0C9
:100330005CEF2AF012000009D8A4A5EF01F000013B
:10034000000E0F6E000E106E1200E806030B0A0D71
:10035000F9CFE8FFF350F92683C00FF084C010F006
:10036000120085C00FF086C010F0120087C00FF099
:1003700088C010F0120089C00FF08AC010F012007F
:10040000EFCFE8FFE806070B0A0DF9CFE8FFF3503E
:10041000F9263CC04EF03DC04FF012003AC04EF0FD
:100420003BC04FF012003EC04EF03FC04FF01200F4
:1004300040C04EF041C04FF0120042C04EF043C0E9
:100440004FF0120044C04EF045C04FF0120046C0BD
:100450004EF047C04FF0120048C04EF049C04FF078
:1004600012000F0B060DF9CFE8FFF350F926BBC2BF
:10047000E8FF1200BCC2E8FF1200BDC2E8FF120094
:10048000BEC2E8FF1200BFC2E8FF1200C0C2E8FF10
:100490001200C1C2E8FF1200C2C2E8FF1200C3C2CC
:1004A000E8FF1200C4C2E8FF1200C5C2E8FF120054
:1004B000C6C2E8FF1200C7C2E8FF1200C8C2E8FFC8
:0E04C0001200C9C2E8FF1200CAC2E8FF120013
:100500000001E806070B0A0DF9CFE8FFF350F926C2
:100510008D510D6E8E510E6E12008F510D6E9051D9
:100520000E6E120091510D6E92510E6E120093518B
:100530000D6E94510E6E120095510D6E96510E6E09
:10054000120097510D6E98510E6E120099510D6E5A
:100550009A510E6E12009B510D6E9C510E6E120040
:100600000001E8BE33EF03F0E806070B0A0DF9CF4F
:10061000E8FFF350F9260D5073270E507423120093
:100620000D5075270E50762312000D5077270E506F
:10063000782312000D5079270E507A2312000D50A6
:100640007B270E507C2312000D507D270E507E23F9
:1006500012000D507F270E50802312000D5081276D
:100660000E5082231200E806070B0A0DF9CFE8FFAF
:10067000F350F9260D50736F0E50746F12000D5029
:10068000756F0E50766F12000D50776F0E50786FA9
:1006900012000D50796F0E507A6F12000D507B6F63
:1006A0000E507C6F12000D507D6F0E507E6F120049
:1006B0000D507F6F0E50806F12000D50816F0E50E5
:1006C000826F1200F2AE12000001010EA16FA1674D
:1006D00067EF03F0120092988088939C819C000140
:1006E0005B6A5C6A640E9DEC0BF092988088000156
:1006F000546A640E9DEC0BF00F018350306E316E26
:10070000326E0F018450336E346E356E0F01999046
:10071000878094969394829681940001000E176EC0
:10072000000E186E0001000E196E000E1A6E000108
:10073000000E1B6E000E1C6E0001000E1D6E000EE2
:100740001E6E0001000E136E000E146E0001000EEE
:10075000156E000E166E0001000EAB6F000EAC6F32
:100760000001000EAD6F000EAE6F0001000EAF6F06
:10077000000EB06F0001000EB16F000EB26F0001ED
:100780005E6A5F6A606BA16BA26BA36BE769E96B42
:100790000201BA6B0101116B0001CC6B3EEC32F02F
:1007A000020100510001A56F040E93EC08F0040E45
:1007B00093EC08F00001C350C56FC450C66F050E1E
:1007C00093EC08F0050E93EC08F00001C350C76FDE
:1007D000C450C86F000EE8CF0DF0E86AE8CF0EF005
:1007E000A8EC0BF0E8CF00F5010EE8CF0DF0E86AB9
:1007F000E8CF0EF0A8EC0BF0E8CF01F5C0EC0CF060
:10080000FA0E9DEC0BF0FA0E9DEC0BF0FA0E9DEC3F
:100810000BF0FA0E9DEC0BF0C8EC08F0B6EC24F0EF
:1008200095EC0EF0A9EC0EF0F28EF28CD08E0F014A
:10083000D89083B6D880D8B023EF04F00A0E9DEC90
:100840000BF00F01D89083B6D880D8B039EF04F000
:100850000F01D89084B2D880D8B034EF04F00A0EDB
:100860009DEC0BF00F01D89084B2D880D8A05BEF3C
:1008700004F082EC1EF00201A50EA76346EF04F01F
:10088000E70EA86346EF04F04AEF04F03EEC32F0C6
:10089000C9EC0BF000C2E8FFFDEC1EF00301AD5106
:1008A0000201A56FE9EC0AF064EC0AF00101F20E16
:1008B000066FA1EC0AF00F01D89084B2D880D8A0BE
:1008C0005BEF04F00A0E9DEC0BF00F01D89084B2A0
:1008D000D880D8A05BEF04F00F01D89084B4D88002
:1008E000D8B078EF04F00A0E9DEC0BF00F01D89011
:1008F00084B4D880D8B08EEF04F00F01D89083B6BE
:10090000D880D8B089EF04F00A0E9DEC0BF00F01EF
:10091000D89083B6D880D8A0BBEF07F00201A0C260
:100920000AF00201FF0E0AB0A56FA561FBEF04F00B
:100930000301A6A1DBEF04F00F0183BEDBEF04F09F
:10094000800E0FEC0DF0000EF86E650EF76EEC0EDB
:10095000F66E75EC0DF0C00E0FEC0DF0000EF86E9B
:10096000650EF76E920EF66E75EC0DF00F01D890D5
:1009700084B4D880D8B0C2EF04F00A0E9DEC0BF01E
:100980000F01D89084B4D880D8B0B6EF04F00F012E
:10099000D89084B4D880D8A0C7EF04F00A0E9DEC9C
:1009A0000BF00F01D89084B4D880D8A0C7EF04F022
:1009B000C80E9DEC0BF00201D1B1E2EF04F0D1A31F
:1009C000FBEF04F0800E00019D6F55EC31F0D890E4
:1009D00025EC27F0D8B0F2EF04F00201FF0EA56F6E
:1009E000FBEF04F0E9EC0AF064EC0AF0A1EC0AF089
:1009F0000A0E9DEC0BF00001010E366EA3C252F000
:100A0000A4C253F00201A25100014D6E59EC23F033
:100A100055EC1FF0FCAE10EF05F00F01939481949C
:100A2000000133B030EF05F0010E366296EF05F0AD
:100A30000001050EE8CF5DF0070E37EC0AF0020E5C
:100A4000366E0001A5510201006329EF05F096EF13
:100A500005F0006FFDEC1EF055EC1FF096EF05F071
:100A6000010E366EFAEC22F0EDEC17F040EC07F0D8
:100A70000201A1A161EF05F00301B6516EEC24F073
:100A8000D8A061EF05F00201B76759EF05F0ABC0E0
:100A900073F0ACC074F0ADC075F0AEC076F0AFC00E
:100AA00077F0B0C078F0B1C079F0B2C07AF061EF01
:100AB00005F0F08CF086A290E868E8CFEEF067EFE2
:100AC00005F0F09CF086A280E86AE8CFEEF0020123
:100AD000A0B186EF05F01FEC17F0D8B486EF05F053
:100AE000ACEC19F03FEC19F079EC1BF00BEC1CF0BE
:100AF0000AEC1AF08FEC21F0ADEC1FF097EC21F02E
:100B0000F0EC1AF00001E9672CEC10F062EC03F055
:100B1000ECEC1CF04EEC0EF00001A26794EF05F037
:100B20000A0EA26FDEEC05F00AEF05F0800E0FEC66
:100B30000DF0000EF86E670EF76E1E0EF66E75EC79
:100B40000DF0C00E0FEC0DF0000EF86E650EF76E96
:100B5000920EF66E75EC0DF071EC1EF0D8A0B3EFAE
:100B600005F030EC25F0EDEC17F0ACEC19F03FECB3
:100B700019F079EC1BF00BEC1CF00AEC1AF08FEC7E
:100B800021F0ADEC1FF097EC21F0F0EC1AF0ECEC5A
:100B90001CF04EEC0EF00AEF05F00001100E0B6E8B
:100BA000C00E0FEC0DF0000EE16E030EE26EE6508B
:100BB00000EC0DF00B2ED7EF05F012000001840EB3
:100BC0000FEC0DF0200E00EC0DF00201520EA5BF4F
:100BD000200E000100EC0DF00601CE516EEC24F069
:100BE000410ED8A0200E00EC0DF00301B2516EECC6
:100BF00024F04D0ED8B02D0E00EC0DF00301B351D2
:100C00006EEC24F04D0ED8B02D0E00EC0DF003016B
:100C1000B4516EEC24F04D0ED8B02D0E00EC0DF05A
:100C2000200E00EC0DF0800E0FEC0DF0B9C20DF0AF
:100C3000BAC20EF00E6A0001640E0F6E000E106E46
:100C400057EC10F013C011F014C012F08BC00DF06F
:100C50008CC00EF013C20FF014C210F057EC10F05D
:100C60001450E8CF13F01550E8CF14F0156A0101C5
:100C700011B14BEF06F000011150135C12501458E3
:100C8000E8AE4BEF06F0C90E00015D6E050E37ECC5
:100C90000AF001011169000105EC0EF0200EE8CF09
:100CA0000AF0300E25640AC025F0255000EC0DF046
:100CB000265000EC0DF02E0E00EC0DF0275000EC4D
:100CC0000DF00301B6516EEC24F0D8A071EF06F0E0
:100CD000800E0FEC0DF000C513F001C514F0DBEC35
:100CE0000DF00201B8AF8AEF06F0B86B000EE8CF46
:100CF0000DF0E86AE8CF0EF000C5E8FFB3EC0BF0AA
:100D0000010EE8CF0DF0E86AE8CF0EF001C5E8FF6C
:100D1000B3EC0BF069EC07F0D8B0B4EF06F07AEC66
:100D200007F0D8B0B4EF06F0BBEC24F0D8B0B4EFC5
:100D300006F08DEC23F00001A351E812D8A4B4EF23
:100D400006F00201A0A1B2EF06F0C00E0FEC0DF00C
:100D5000000EF86E650EF76EAC0EF66E75EC0DF0CB
:100D6000B4EF06F0CDEC05F0000133B4CFEF06F0A0
:100D700035A4CFEF06F03594010E5D6E050E37EC0D
:100D80000AF000015466CEEF06F0542ABEC358F0B4
:100D9000BFC359F0CA6BCB6BCFEF06F0540600010E
:100DA00054A002EF07F0596602EF07F03B0E5A62BB
:100DB000E1EF06F0050E5D6E0A0E37EC0AF002EF69
:100DC00007F01E0E5A62ECEF06F0030E5D6E0A0E7F
:100DD00037EC0AF002EF07F00A0E5A62F7EF06F05E
:100DE000010E5D6E0A0E37EC0AF002EF07F0060EF8
:100DF0005A6002EF07F0010E5D6E0A0E37EC0AF042
:100E000002EF07F07F0E5A6E5650CE6F5750CF6FDD
:100E1000010E54622BEF07F058505910D8B41AEF56
:100E200007F05850CE6F5950CF6F000E0301BD63CD
:100E30002BEF07F0020E0301BD5DD8B427EF07F0DA
:100E40000001CA51CE6FCB51CF6F2BEF07F0E86A8C
:100E50000001CE6FCF6F00018B0E0FEC0DF0CF5164
:100E6000E8CF13F0146A156A166AD3EC0DF03A0E47
:100E700000EC0DF0CE51E8CF13F0D3EC0DF01200E2
:100E80000301C0516EEC24F0D8A066EF07F0030117
:100E9000000EC16563EF07F000017ABF66EF07F04F
:100EA0000301C15100010D6E0E6A00010A0E0F6EA2
:100EB000000E106E57EC10F07951135E7A51145CED
:100EC000D8B066EF07F00001E76912000001E76B98
:100ED0001200D8900001CCAF1200C00E0FEC0DF044
:100EE000000EF86E660EF76E580EF66E75EC0DF08D
:100EF000D88012000D0E93EC08F00D0E93EC08F064
:100F000069C00DF06AC00EF0A9C20FF0AAC210F0BD
:100F100057EC10F000011450136E1550146E16505B
:100F2000156E166A05EC0EF00001255026100F0B09
:100F3000D890D8B41200C00E0FEC0DF0000EF86E71
:100F4000660EF76E460EF66E75EC0DF0CB0E0FECDE
:100F50000DF00001255000EC0DF0265000EC0DF0D6
:100F60002E0E00EC0DF0275000EC0DF0285000EC98
:100F70000DF0D88012000F01D89084B4D880D8A08A
:100F8000BBEF07F00A0E9DEC0BF00F01D89084B474
:100F9000D880D8A0BBEF07F00F01D89083B6D880D7
:100FA000D8A0CCEF07F00A0E9DEC0BF00F01D89003
:100FB00083B6D880D8A0CCEF07F0800E0FEC0DF0F0
:100FC0000F01835092EC0DF00F01845092EC0DF064
:100FD000C00E0FEC0DF00F01865092EC0DF00F01DA
:100FE000875092EC0DF00F01835082868184E8B027
:100FF0008296E8B281948098E8B48088320E9DECA5
:101000000BF00F01D89084B4D880D8B00DEF08F061
:101010000A0E9DEC0BF00F01D89084B4D880D8B0A4
:10102000DDEF07F00F01D89084B4D880D8A012EF7C
:1010300008F00A0E9DEC0BF00F01D89084B4D88014
:10104000D8A012EF08F0C00E0FEC0DF0000EF86EF5
:10105000650EF76E020EF66E75EC0DF000010D6A6E
:10106000800E0FEC0DF0000EF86E650EF76E380E68
:10107000F66E75EC0DF0870E0FEC0DF000010D50C3
:101080009FEC0DF093EC08F08C0E0FEC0DF00F01BF
:10109000C4CFE8FF9FEC0DF00F01C3CFE8FF9FEC3A
:1010A0000DF0320E9DEC0BF00F01D89084B4D88077
:1010B000D8B060EF08F00A0E9DEC0BF00F01D8904D
:1010C00084B4D880D8B030EF08F00F01D89084B441
:1010D000D880D8A065EF08F00A0E9DEC0BF00F0148
:1010E000D89084B4D880D8A065EF08F000010D2A0C
:1010F0000C0E0D6430EF08F0DDEF07F00001136A0D
:10110000146A156A166A0A6E0B6A0A5093EC08F0A4
:101110000001C3501326C4501422D8B0152A0B2E38
:1011200085EF08F012000A6EA10EC06E000EC16EAF
:101130000AC0E8FF31EC02F0E8AEC188E89EE8445E
:10114000E844C26EC2800000C282C2B2A5EF08F0BD
:101150000001C3CF69F0C4CF6AF00AC0E8FF1200F3
:101160000F01C282C2B2B2EF08F00001C35069277A
:10117000C4506A23120093EC08F0B0EC08F0B0EC15
:1011800008F0B0EC08F000016A336A9F693312007E
:1011900000014C6A566A576A280EE8CF55F00001E4
:1011A000900E526E010E536E0001900E4E6E010EA7
:1011B0004F6E506A516A100E0001E8CF4DF0386A48
:1011C0003A6A3C6A3E6A406A426A446A466A486AC7
:1011D0004A6A080EE8CF39F0E8CF3BF0E8CF3DF09F
:1011E000E8CF3FF0E8CF41F0E8CF43F0E8CF45F05B
:1011F000E8CF47F0E8CF49F0E8CF4BF0979E858ED7
:10120000000152500F01E8CFBBFF010153500F0105
:10121000E8CFBCFF0A0E0F01E8CFBAFF0F01A08094
:101220000F019E900F01080EE8CFB1FFB1801200B0
:101230000001EEA1857E0201BAAF22EF09F08770AE
:101240002AEF09F00001E5B129EF09F087802AEFC4
:1012500009F087900001BBCFE8FF4E26BCCFE8FF26
:101260004F224EC0E8FFE8CFBBFF4FC0E8FFE8CFFA
:10127000BCFF0001E86A4C64A1EC09F000014C2AB3
:101280004CC0E8FFFE0B4D6057EF09F04C6A500E62
:10129000E8CF4EF050C0E8FF4E5EC30EE8CF4FF0EF
:1012A00051C0E8FF4F5A506A516A9EEF09F04CA0B6
:1012B0006CEF09F052C0E8FFE8CF4EF053C0E8FFF2
:1012C000E8CF4FF0BAC2E8FF0001E5814C6298EF29
:1012D00009F0E59198EF09F0120E4C6284EF09F0E5
:1012E00050C0E8FFE8CF4EF051C0E8FFE8CF4FF024
:1012F0004F324E324F324E324F324E324F324E32EA
:101300000F0E4F1698EF09F0040EE8CFEAFF000E1B
:10131000E8CFE9FF4CC0E8FFE830E89EE804E926A2
:1013200000EC02F052C0E8FF4E5E53C0E8FF4F5A97
:101330004EC0E8FF50264FC0E8FF51220F01A19098
:10134000120083EC0EF08DEC0EF00001010E3662FF
:10135000B0EF09F000018286BDB18296FF0EBD6F2D
:1013600087900301CDBFB8EF09F0859EB9EF09F072
:10137000858E0001552EFFEF09F0B9EC24F0000135
:1013800054A0EFEF09F00001FF0EE763EFEF09F063
:1013900058C0E8FF5910D8B4E7EF09F05866D4EF09
:1013A00009F03C0E586E5906580658505A6E030103
:1013B000E86ABD11D8B4E7EF09F0000158505910A0
:1013C000D8B4E7EF09F0CA6BCB6BEFEF09F000017F
:1013D000CA2B3C0ECA63EFEF09F0CA6BCB2B280E69
:1013E000E8CF55F0562A3C0E5662FFEF09F0566AD8
:1013F000572A0501002BD8B4012B0201B86902015C
:10140000A1A108EF0AF0530EB5EC0EF00001A86B95
:10141000000183CFE8FF311AD8A4306E316E30C09E
:10142000E8FF3212000184CFE8FF341AD8A4336EEB
:10143000346E33C0E8FF351200015E665E065F66FB
:101440005F0660676007A167A107A267A207A3679D
:10145000A3075C662DEF0AF012005C2E1200807864
:101460005D4E12005BC0E8FFE8CF5CF01200E8CFF1
:101470005BF0E8CF5CF08098120000010ABE44EFF8
:101480000AF0819E45EF0AF0818E828A829A0A468E
:101490000B2E3DEF0AF012000201AD510A6E080E4C
:1014A0000B6E3DEC0AF00201AC510A6E080E0B6E99
:1014B0003DEC0AF00201AB510A6E080E0B6E3DECDA
:1014C0000AF08686869612000BC113F00CC114F048
:1014D0000DC115F009C117F00AC118F05BEC11F04D
:1014E0000201A55101010F03F35000011326D8B0EA
:1014F000142AD8B0152A0101006B016B026B0001A0
:101500001350E846E846E880E8921F0B13B6E88ED1
:101510000101006F000113361436153613361436E8
:101520001536133614361536133614361536145050
:101530000101016F000115501F0B01011009026F1D
:10154000120064EC0AF0010108510A6E080E0B6EDD
:101550003DEC0AF0010107510A6E080E0B6E3DECDE
:101560000AF0010106510A6E080E0B6E3DEC0AF0FE
:1015700086868696010105510A6E080E0B6E3DECBB
:101580000AF0010104510A6E080E0B6E3DEC0AF0E0
:10159000010103510A6E080E0B6E3DEC0AF08686BF
:1015A0008696010102510A6E080E0B6E3DEC0AF0A0
:1015B000010101510A6E080E0B6E3DEC0AF00101AB
:1015C00000510A6E080E0B6E3DEC0AF08686869678
:1015D00012000F01939E949A939C819C819E829A03
:1015E000989686960201D1A118EF0BF0D1B318EFAF
:1015F0000BF004C206F105C207F106C208F101C2F0
:1016000003F102C204F103C205F10101700E0B6F78
:10161000C60E0C6F000E0D6F0101140E096F000E47
:101620000A6F01010E6B0A0E106F010E0F6F120090
:101630000201D1B13EEF0BF0D1A33EEF0BF00AC295
:1016400006F10BC207F10CC208F107C203F108C290
:1016500004F109C205F101016C0E0B6FCF0E0C6F86
:10166000000E0D6F0101640E096F000E0A6F01017B
:101670000E6B080E106F010E0F6F12000201D1B138
:1016800065EF0BF0D1B365EF0BF010C206F111C29C
:1016900007F112C208F10DC203F10EC204F10FC22C
:1016A00005F101014A0E0B6F190E0C6F010E0D6F43
:1016B00001010A0E096F000E0A6F01010B0E0E6F79
:1016C000320E106F020E0F6F1200120087B284EFFD
:1016D0000BF0D5AE76EF0BF0D6CFC1F0D7CFC2F07E
:1016E0000001C32BD8B4C42BF09012000001C351E9
:1016F000C411F090D8A41200E86AE8CFD7FFE8CF71
:10170000D6FFD58EF0901200F17AF0AC96EF0BF088
:101710000301CDA192EF0BF0F1AA859EF1BA858E5F
:1017200096EF0BF0F1AA858EF1BA859EF09012002B
:101730000000E82E98EF0BF012000A6EFA0E98ECFB
:101740000BF0FA0E98EC0BF00A2E9EEF0BF0120045
:101750000EC0E8FFAA6E0DC0E8FFA96EA69EA69C6B
:10176000A680A8501200A86E0EC0E8FFAA6E0DC099
:10177000E8FFA96EA69EA69CA684F29E550EA76EB3
:10178000AA0EA76EA682F28EA1A8C4EF0BF0A198B4
:101790001200800E0FEC0DF0000EF86E650EF76E65
:1017A000FE0EF66E75EC0DF0C00E0FEC0DF0000E97
:1017B000F86E650EF76E800EF66E75EC0DF06EEC41
:1017C00027F0D8A009EF0CF0C00E0FEC0DF0000EC2
:1017D000F86E660EF76E100EF66E75EC0DF03EECC0
:1017E00032F097EC1EF00001600E9E6F00C2E8FF21
:1017F00028EC1FF00201002B0301072B3A0E0763B0
:1018000005EF0CF0062B300E076F00019E2FF6EF50
:101810000BF082EC1EF000C2E8FFFDEC1EF012009F
:1018200000011550F86E1450F76E1350F66E00015B
:101830000E50E26E0D50E16E0900F550E66E0A069C
:101840000900F550E66E0A2E1CEF0CF012000001A4
:101850001550F86E1450F76E1350F66EA68EA69CB7
:10186000A684A688F29E550EA76EAA0EA76EA68223
:101870000000F28E0001400E1326000E14221522E5
:101880000A2E27EF0CF0120062EC03F00001155055
:10189000F86E1450F76E1350F66EA68EA69CA684B2
:1018A000A688F29E550EA76EAA0EA76EA682F28E8D
:1018B0000A0000010E50E26E0D50E16E400E0B6EFC
:1018C000E6CFE8FFF56E0F000B2EFAD7A68EA69C8A
:1018D000A684F29E550EA76EAA0EA76EA682F28E61
:1018E000A6940001400E1326000E142215220001BA
:1018F000400E0D26000E0E220A2E44EF0CF01200B0
:1019000000011550F86E1450F76E1350F66EA68E47
:10191000A69CA684A688F29E550EA76EAA0EA76E58
:10192000A6820000F28E0A00080E0B6E00010E5017
:10193000E26E0D50E16E080E0C6EE6CFE8FFF56E1C
:101940000F000C2EFAD7A68EA69CA684F29E550EEA
:10195000A76EAA0EA76EA6820000F28E0B2EEBD702
:10196000A6940001400E1326000E14221522000139
:10197000400E0D26000E0E220A2E80EF0CF01200F3
:101980000F019A6A886A9396939A93988186818ABE
:101990008188140E9DEC0BF0380E0FEC0DF0050E47
:1019A0009DEC0BF0380E0FEC0DF0010E9DEC0BF0E2
:1019B000380E0FEC0DF0010E9DEC0BF0380E0FEC15
:1019C0000DF0060E0FEC0DF00E0E0FEC0DF0010EEB
:1019D0000FEC0DF0800E0FEC0DF0800E0FEC0DF003
:1019E000650EF76E140EF66E75EC0DF0C00E0FEC72
:1019F0000DF0650EF76E260EF66E75EC0DF012000A
:101A00001EEC0DF032EC0DF0818A81980000000090
:101A100081860000000081960000000012001EEC8C
:101A20000DF032EC0DF0819A819800000000818663
:101A300000000000819600000000120025EC0DF06F
:101A4000D8B01EEF0DF09A6A12009A688188819AC8
:101A500000000000818600000000D89088BED88079
:101A600081961200886E12001010101010101010C5
:101A700018181818181818181C1C1C1C1C1C1C1CC6
:101A80001E1E1E1E1E1E1E1E01010101010101015E
:101A900003030303030303030707070707070707F6
:101AA0000F0F0F0F0F0F0F0F800E0FEC0DF00DC06B
:101AB000F6FF0EC0F7FFF86A75EC0DF01200C00ECD
:101AC0000FEC0DF00DC0F6FF0EC0F7FFF86A75ECD5
:101AD0000DF01200C00E0FEC0DF0CEC0F6FFCFC01F
:101AE000F7FFF86A75EC0DF01200100E78EF0DF0AC
:101AF0000A6E0900F5CFE8FFE812D8B491EF0DF0B7
:101B000000EC0DF00A4E91EF0DF00900F5CFE8FF63
:101B1000E812D8B491EF0DF000EC0DF00A2E79EF39
:101B20000DF012000A6E080E0B6E300E0ABE310E5A
:101B300000EC0DF00A360B2E95EF0DF012000A6E38
:101B40003A0E0B6E0AC0E8FFF00BE842E842E842AA
:101B5000E84230090B64070F00EC0DF00AC0E8FF03
:101B60000F0B30090B64070F00EC0DF00AC0E8FF03
:101B7000120005EC0EF0255000EC0DF0265000ECA4
:101B80000DF0275000EC0DF0285000EC0DF029501E
:101B900000EC0DF0120005EC0EF0BEEF0DF005ECC0
:101BA0000EF0C1EF0DF005EC0EF0C4EF0DF005ECFA
:101BB0000EF0C7EF0DF005EC0EF0EFEC0DF0255038
:101BC00000EC0DF0265000EC0DF0275000EC0DF06D
:101BD000285000EC0DF0295000EC0DF0120000012F
:101BE000300E25621200200E256E300E2662120085
:101BF000200E266E300E27621200200E276E300E49
:101C000028621200200E286E12000001196A1A6A5A
:101C1000100E176E270E186E5BEC11F0300E1310BD
:101C2000256E1BC013F01CC014F01DC015F01EC0A3
:101C300016F0196A1A6AE80E176E030E186E5BEC3E
:101C400011F0300E1310266E1BC013F01CC014F0E0
:101C50001DC015F01EC016F0196A1A6A640E176EC0
:101C6000000E186E5BEC11F0300E1310276E1BC0C7
:101C700013F01CC014F01DC015F01EC016F0196A38
:101C80001A6A0A0E176E000E186E5BEC11F0300E19
:101C90001310286E300E1B10296E12000001310E39
:101CA000376257EF0EF082EC1EF081EF0EF0320E2D
:101CB000376261EF0EF000C2E8FFFDEC1EF081EF2D
:101CC0000EF0330E376269EF0EF097EC1EF081EFE5
:101CD0000EF0340E376271EF0EF000C2E8FF28EC10
:101CE0001FF0350E376281EF0EF00001FF0E0D6E12
:101CF000030E0E6EE8CF0EF0FF0EB3EC0BF081EF8B
:101D00000EF0376A12000F01ABA21200AB98AB883D
:101D10000F01AE500001616B12000F016BA21200A7
:101D20006B986B880F016E5012000C0EE8CFAFFF5E
:101D3000220EE8CFACFF900EE8CFABFF0001616B45
:101D40009F9A9D8A1200ACA2A3EF0EF0E8CFADFFE0
:101D50001200000EE8CF6FFF220EE8CF6CFF900E4E
:101D6000E8CF6BFFA59AA38A12006CA2B5EF0EF024
:101D7000E8CF6DFF1200E1CF21F0E2CF22F00001A9
:101D800065C0E1FF000164C0E2FF686BACA2C6EF72
:101D90000EF0E6CFE8FF00016827E8CFADFF0001B5
:101DA000662FC6EF0EF021C0E1FF22C0E2FF120055
:101DB000E1CF21F0E2CF22F0000165C0E1FF000198
:101DC00064C0E2FF686B0001050E5E6EE86A5E6447
:101DD000F7EF0EF09EAAE7EF0EF0AECFE8FFE8CFE8
:101DE000E6FF000168270001662FE3EF0EF021C037
:101DF000E1FF22C0E2FF12009EAA12000001000EC5
:101E000061630FEF0FF0AECFE8FFE8CF62F0550E41
:101E100062631200280EE8CF5FF0612B1200010E02
:101E2000616319EF0FF0AECFE8FFE8CF63F0612BED
:101E30001200020E616323EF0FF0AECFE8FFE8CF90
:101E400064F0612B1200030E61632DEF0FF0AECF33
:101E5000E8FFE8CF65F0612B1200040E616336EFF6
:101E60000FF0AECFE8FFE8CF66F0612B050E61639F
:101E700042EF0FF0010E636340EF0FF0D8EC0EF06D
:101E8000612B1200060E616365EF0FF0AECFE8FF25
:101E9000E8CF67F0020E636356EF0FF0BBEC0EF075
:101EA00068C0E8FFA3EC0EF0616B120068C0E8FFA9
:101EB000676360EF0FF00C0EA3EC0EF0616B120085
:101EC0000D0EA3EC0EF0616B1200616B1200A4AA60
:101ED00012006ECFE8FF0201A1B19BEF0FF0530A91
:101EE000D8A412000201A0A1120000010F0E741567
:101EF0001009B5EC0EF073C0E8FFB5EC0EF0000170
:101F00000F0E76152009B5EC0EF07551B5EC0EF0FC
:101F100000010F0E78153009B5EC0EF07751B5ECD5
:101F20000EF000010F0E7A154009B5EC0EF0795154
:101F3000B5EC0EF012000001A8B1A2EF0FF0AA6FED
:101F4000A82B1200A96FA82B020EA863BBEF0FF0FD
:101F5000AA51F00B100AD8A400EF10F00F0EAA1728
:101F6000AAA7B5EF0FF0F00EAA13A9C0ABF0AAC054
:101F7000ACF000EF10F0040EA863D2EF0FF0AA51FE
:101F8000F00B200AD8A400EF10F00F0EAA17AAA792
:101F9000CCEF0FF0F00EAA13A9C0ADF0AAC0AEF0BE
:101FA00000EF10F0060EA863E9EF0FF0AA51F00B56
:101FB000300AD8A400EF10F00F0EAA17AAA7E3EF7B
:101FC0000FF0F00EAA13A9C0AFF0AAC0B0F000EF56
:101FD00010F0080EA86300EF10F0AA51F00B400AB1
:101FE000D8A400EF10F00F0EAA17AAA7FAEF0FF06F
:101FF000F00EAA13A9C0B1F0AAC0B2F000EF10F021
:1020000012000C0E0F016F6E220E6C6E900EE8CF58
:102010006BFF12000001E80E0D26030E0E22780E53
:102020000D5C070E0E58D8A019EF10F0EF0E20EF40
:1020300010F00E320D320E320D320E320D320D50C6
:10204000B5EF0EF0BC0E0D5C030E0E58D8A01BEFC2
:1020500010F0EF0E20EF10F0F00EB5EC0EF0800E49
:10206000B5EC0EF073C00DF074C00EF00AEC10F079
:1020700075C00DF076C00EF00AEC10F077C00DF0D0
:1020800078C00EF00AEC10F079C00DF07AC00EF0B6
:1020900022EC10F07BC00DF07CC00EF022EC10F0B2
:1020A0007DC00DF07EC00EF022EC10F0120068EC46
:1020B00010F010AE60EF10F00D50155E0E50165A75
:1020C0000EAE67EF10F00F50155E1050165A12004A
:1020D0000001136A146A156A166A0F500D02F3CFD5
:1020E00013F0F4CF14F00F500E02F3501426F450F6
:1020F0001522D8B0162A10500D02F3501426F450B1
:102100001522D8B0162A10500E02F3501526F4509E
:10211000162212000001246A1B6A14501310D8B44E
:10212000000C14501718E8BE241EA46B000E17AE46
:102130009CEF10F0171E172A14AEA3EF10F0131E19
:10214000141E132A142214501710E8BE2FEF11F09A
:1021500017501B5E143614341B3617501B261436CA
:1021600014341B36175014B01B5E14A01B261436F3
:1021700014341B36175014B01B5E14A01B261436E3
:1021800014341B36175014B01B5E14A01B261436D3
:1021900014341B36175014B01B5E14A01B261436C3
:1021A00014341B36175014B01B5E14A01B261436B3
:1021B00014341B36175014B01B5E14A01B261436A3
:1021C00013341B36175014B01B5E14A01B26133695
:1021D00013341B36175013B01B5E13A01B26133687
:1021E00013341B36175013B01B5E13A01B26133677
:1021F00013341B36175013B01B5E13A01B26133667
:1022000013341B36175013B01B5E13A01B26133656
:1022100013341B36175013B01B5E13A01B26133646
:1022200013341B36175013B01B5E13A01B26133636
:1022300013341B36175013B01B5E13A01B26133626
:1022400013A01B26A4B14DEF11F024AE000C131EF9
:10225000141EE86A132A14221B1E1B2A000C17AE38
:1022600048EF11F014BE44EF11F0E8CF9DF0135089
:10227000E8CF1BF01B9E133614361450E8CF13F032
:102280009D51146A25EF11F0136A132A146A000C89
:10229000141E131EA42BA8EF10F01B2A17501B624C
:1022A00025EF11F01B6A000E132A142214AE25EF3D
:1022B00011F02388FF0C0001246A1C6A1B6A155068
:1022C00014101310D8B4000C15501818E8BE241EB2
:1022D000A46B000E18AE71EF11F0171E181E172A0E
:1022E000182215AE7AEF11F0131E141E151E132AB4
:1022F0001422152215501810E8BE04EF13F01750E1
:102300001B5E18501C5A153615341B361C361750D8
:102310001B2618501C22153615341B361C36175038
:1023200015A098EF11F01B5E18501C5A9BEF11F08E
:102330001B2618501C22153615341B361C36175018
:1023400015A0A8EF11F01B5E18501C5AABEF11F04E
:102350001B2618501C22153615341B361C361750F8
:1023600015A0B8EF11F01B5E18501C5ABBEF11F00E
:102370001B2618501C22153615341B361C361750D8
:1023800015A0C8EF11F01B5E18501C5ACBEF11F0CE
:102390001B2618501C22153615341B361C361750B8
:1023A00015A0D8EF11F01B5E18501C5ADBEF11F08E
:1023B0001B2618501C22153615341B361C36175098
:1023C00015A0E8EF11F01B5E18501C5AEBEF11F04E
:1023D0001B2618501C22153614341B361C36175079
:1023E00015A0F8EF11F01B5E18501C5AFBEF11F00E
:1023F0001B2618501C22143614341B361C3617505A
:1024000014A008EF12F01B5E18501C5A0BEF12F0CC
:102410001B2618501C22143614341B361C36175039
:1024200014A018EF12F01B5E18501C5A1BEF12F08C
:102430001B2618501C22143614341B361C36175019
:1024400014A028EF12F01B5E18501C5A2BEF12F04C
:102450001B2618501C22143614341B361C361750F9
:1024600014A038EF12F01B5E18501C5A3BEF12F00C
:102470001B2618501C22143614341B361C361750D9
:1024800014A048EF12F01B5E18501C5A4BEF12F0CC
:102490001B2618501C22143614341B361C361750B9
:1024A00014A058EF12F01B5E18501C5A5BEF12F08C
:1024B0001B2618501C22143614341B361C36175099
:1024C00014A068EF12F01B5E18501C5A6BEF12F04C
:1024D0001B2618501C22143613341B361C3617507A
:1024E00014A078EF12F01B5E18501C5A7BEF12F00C
:1024F0001B2618501C22133613341B361C3617505B
:1025000013A088EF12F01B5E18501C5A8BEF12F0CC
:102510001B2618501C22133613341B361C3617503A
:1025200013A098EF12F01B5E18501C5A9BEF12F08C
:102530001B2618501C22133613341B361C3617501A
:1025400013A0A8EF12F01B5E18501C5AABEF12F04C
:102550001B2618501C22133613341B361C361750FA
:1025600013A0B8EF12F01B5E18501C5ABBEF12F00C
:102570001B2618501C22133613341B361C361750DA
:1025800013A0C8EF12F01B5E18501C5ACBEF12F0CC
:102590001B2618501C22133613341B361C361750BA
:1025A00013A0D8EF12F01B5E18501C5ADBEF12F08C
:1025B0001B2618501C22133613341B361C3617509A
:1025C00013A0E8EF12F01B5E18501C5AEBEF12F04C
:1025D0001B2618501C22133613B0F3EF12F01750BD
:1025E0001B2618501C22A4B128EF13F024AE000CB7
:1025F000131E141E151E000E132A142215221B1E54
:102600001C1E1B2A1C22000C18AE22EF13F015BE54
:102610001DEF13F0E8CF9DF01450E8CF1CF01350DD
:10262000E8CF1BF01C9E143615361550E8CF13F07A
:102630009D51156A146AF6EF12F0136A132A146A90
:10264000156A000C151E141E131EA42B7FEF11F02B
:102650001B2AE86A1C2217501B62F6EF12F0185072
:102660001C62F6EF12F01C6A1B6A000E132A142279
:10267000152215AEF6EF12F02388FF0C1E6A1D6AB4
:102680001C6A1B6A16341B361C361D361E36175044
:102690001B5E18501C5A19501D5A1A501E5AA46A13
:1026A000A45B163616341B361C361D361E36A43770
:1026B000175016A067EF13F01B5E18501C5A1950E4
:1026C0001D5A1A501E5AE86AA45B70EF13F01B26BD
:1026D00018501C2219501D221A501E22E86AA423E9
:1026E000163616341B361C361D361E36A4371750C8
:1026F00016A086EF13F01B5E18501C5A19501D5A75
:102700001A501E5AE86AA45B8FEF13F01B2618506C
:102710001C2219501D221A501E22E86AA4231636C4
:1027200016341B361C361D361E36A437175016A01D
:10273000A5EF13F01B5E18501C5A19501D5A1A5061
:102740001E5AE86AA45BAEEF13F01B2618501C2239
:1027500019501D221A501E22E86AA4231636163478
:102760001B361C361D361E36A437175016A0C4EF74
:1027700013F01B5E18501C5A19501D5A1A501E5A3D
:10278000E86AA45BCDEF13F01B2618501C221950E9
:102790001D221A501E22E86AA423163616341B3650
:1027A0001C361D361E36A437175016A0E3EF13F063
:1027B0001B5E18501C5A19501D5A1A501E5AE86AAE
:1027C000A45BECEF13F01B2618501C2219501D229D
:1027D0001A501E22E86AA423163616341B361C36FD
:1027E0001D361E36A437175016A002EF14F01B5EDC
:1027F00018501C5A19501D5A1A501E5AE86AA45BE8
:102800000BEF14F01B2618501C2219501D221A50D1
:102810001E22E86AA423163616341B361C361D36D3
:102820001E36A437175016A021EF14F01B5E185067
:102830001C5A19501D5A1A501E5AE86AA45B2AEFF6
:1028400014F01B2618501C2219501D221A501E224B
:10285000E86AA423163615341B361C361D361E3680
:10286000A437175016A040EF14F01B5E18501C5AE6
:1028700019501D5A1A501E5AE86AA45B49EF14F009
:102880001B2618501C2219501D221A501E22E86ABD
:10289000A423153615341B361C361D361E36A437B8
:1028A000175015A05FEF14F01B5E18501C5A1950FA
:1028B0001D5A1A501E5AE86AA45B68EF14F01B26D2
:1028C00018501C2219501D221A501E22E86AA423F7
:1028D000153615341B361C361D361E36A4371750D8
:1028E00015A07EEF14F01B5E18501C5A19501D5A8B
:1028F0001A501E5AE86AA45B87EF14F01B26185082
:102900001C2219501D221A501E22E86AA4231536D3
:1029100015341B361C361D361E36A437175015A02D
:102920009DEF14F01B5E18501C5A19501D5A1A5076
:102930001E5AE86AA45BA6EF14F01B2618501C224E
:1029400019501D221A501E22E86AA4231536153488
:102950001B361C361D361E36A437175015A0BCEF8B
:1029600014F01B5E18501C5A19501D5A1A501E5A4A
:10297000E86AA45BC5EF14F01B2618501C221950FE
:102980001D221A501E22E86AA423153615341B3660
:102990001C361D361E36A437175015A0DBEF14F079
:1029A0001B5E18501C5A19501D5A1A501E5AE86ABC
:1029B000A45BE4EF14F01B2618501C2219501D22B2
:1029C0001A501E22E86AA423153615341B361C360D
:1029D0001D361E36A437175015A0FAEF14F01B5EF3
:1029E00018501C5A19501D5A1A501E5AE86AA45BF6
:1029F00003EF15F01B2618501C2219501D221A50E7
:102A00001E22E86AA423153615341B361C361D36E3
:102A10001E36A437175015A019EF15F01B5E18507D
:102A20001C5A19501D5A1A501E5AE86AA45B22EF0C
:102A300015F01B2618501C2219501D221A501E2258
:102A4000E86AA423153614341B361C361D361E3690
:102A5000A437175015A038EF15F01B5E18501C5AFC
:102A600019501D5A1A501E5AE86AA45B41EF15F01E
:102A70001B2618501C2219501D221A501E22E86ACB
:102A8000A423143614341B361C361D361E36A437C8
:102A9000175014A057EF15F01B5E18501C5A195010
:102AA0001D5A1A501E5AE86AA45B60EF15F01B26E7
:102AB00018501C2219501D221A501E22E86AA42305
:102AC000143614341B361C361D361E36A4371750E8
:102AD00014A076EF15F01B5E18501C5A19501D5AA1
:102AE0001A501E5AE86AA45B7FEF15F01B26185097
:102AF0001C2219501D221A501E22E86AA4231436E3
:102B000014341B361C361D361E36A437175014A03D
:102B100095EF15F01B5E18501C5A19501D5A1A508B
:102B20001E5AE86AA45B9EEF15F01B2618501C2263
:102B300019501D221A501E22E86AA4231436143498
:102B40001B361C361D361E36A437175014A0B4EFA2
:102B500015F01B5E18501C5A19501D5A1A501E5A57
:102B6000E86AA45BBDEF15F01B2618501C22195013
:102B70001D221A501E22E86AA423143614341B3670
:102B80001C361D361E36A437175014A0D3EF15F08F
:102B90001B5E18501C5A19501D5A1A501E5AE86ACA
:102BA000A45BDCEF15F01B2618501C2219501D22C7
:102BB0001A501E22E86AA423143614341B361C361D
:102BC0001D361E36A437175014A0F2EF15F01B5E09
:102BD00018501C5A19501D5A1A501E5AE86AA45B04
:102BE000FBEF15F01B2618501C2219501D221A50FD
:102BF0001E22E86AA423143614341B361C361D36F4
:102C00001E36A437175014A011EF16F01B5E185093
:102C10001C5A19501D5A1A501E5AE86AA45B1AEF22
:102C200016F01B2618501C2219501D221A501E2265
:102C3000E86AA423143613341B361C361D361E36A0
:102C4000A437175014A030EF16F01B5E18501C5A12
:102C500019501D5A1A501E5AE86AA45B39EF16F033
:102C60001B2618501C2219501D221A501E22E86AD9
:102C7000A423133613341B361C361D361E36A437D8
:102C8000175013A04FEF16F01B5E18501C5A195026
:102C90001D5A1A501E5AE86AA45B58EF16F01B26FC
:102CA00018501C2219501D221A501E22E86AA42313
:102CB000133613341B361C361D361E36A4371750F8
:102CC00013A06EEF16F01B5E18501C5A19501D5AB7
:102CD0001A501E5AE86AA45B77EF16F01B261850AC
:102CE0001C2219501D221A501E22E86AA4231336F2
:102CF00013341B361C361D361E36A437175013A04E
:102D00008DEF16F01B5E18501C5A19501D5A1A50A0
:102D10001E5AE86AA45B96EF16F01B2618501C2278
:102D200019501D221A501E22E86AA42313361334A8
:102D30001B361C361D361E36A437175013A0ACEFB9
:102D400016F01B5E18501C5A19501D5A1A501E5A64
:102D5000E86AA45BB5EF16F01B2618501C22195028
:102D60001D221A501E22E86AA423133613341B3680
:102D70001C361D361E36A437175013A0CBEF16F0A5
:102D80001B5E18501C5A19501D5A1A501E5AE86AD8
:102D9000A45BD4EF16F01B2618501C2219501D22DC
:102DA0001A501E22E86AA423133613341B361C362D
:102DB0001D361E36A437175013A0EAEF16F01B5E1F
:102DC00018501C5A19501D5A1A501E5AE86AA45B12
:102DD000F3EF16F01B2618501C2219501D221A5012
:102DE0001E22E86AA423133613341B361C361D3604
:102DF0001E36A437175013A009EF17F01B5E1850AA
:102E00001C5A19501D5A1A501E5AE86AA45B12EF38
:102E100017F01B2618501C2219501D221A501E2272
:102E2000E86AA423133613B01EEF17F017501B26C1
:102E300018501C2219501D221A501E22000C0F017E
:102E4000D89083B6D880D8B02BEF17F00A0E9DEC3F
:102E50000BF00F01D89083B6D880D8B0A1EF17F04F
:102E60000F01D89084B2D880D8B03CEF17F00A0E8A
:102E70009DEC0BF00F01D89084B2D880D8B0A1EFB0
:102E800017F00001CC6763EF17F00001CC69030174
:102E900032C30DF033C30EF00001E80E0F6E030EC7
:102EA000106E57EC10F014C01CF115C01DF1030199
:102EB000345101011C270301355101011D2334C385
:102EC0001AF135C31BF1A4EC29F0D8B074EF17F058
:102ED000D8A47BEF17F001011A07D8A01B071A0727
:102EE000D8A01B077BEF17F001011A2BD8B41B2BBE
:102EF0001A2BD8B41B2B1CC10DF01DC10EF0010103
:102F00001A5100010D5E01011B5100010E5A000112
:102F1000000E0F6E010E106E57EC10F00001E80E5F
:102F2000176E030E186E5BEC11F013C032F314C071
:102F300033F31AC134F31BC135F30AEC1AF0D88409
:102F400012000001CC67A7EF17F0D8941200CC6BE9
:102F500072EC1FF0D894120000016951E8CF0DF017
:102F60006A51E8CF0EF06D510D5E6E510E5AD8A029
:102F7000C9EF17F06B51E8CF0FF06C51E8CF10F0AC
:102F800057EC10F01450E8CF71F01550E8CF72F004
:102F900012006F51E8CF0FF07051E8CF10F057ECEE
:102FA00010F01450E8CF71F01550E8CF72F0120015
:102FB00069C00DF06AC00EF06D510D5E6E510E5A73
:102FC0006BC00FF06CC010F057EC10F01450E8CF4D
:102FD00071F01550E8CF72F01200040E93EC08F077
:102FE000040EBBEC08F015C26BF016C26CF017C2F1
:102FF0006DF018C26EF019C26FF01AC270F0ACEC2E
:1030000017F071C034F172C035F171C073F072C045
:1030100074F0050E93EC08F0050EBBEC08F01BC233
:103020006BF01CC26CF01DC26DF01EC26EF01FC2B0
:103030006FF020C270F0ACEC17F071C036F172C0C6
:1030400037F171C075F072C076F0060E93EC08F09F
:10305000060EBBEC08F021C26BF022C26CF023C25A
:103060006DF024C26EF025C26FF026C270F0ACEC99
:1030700017F071C038F172C039F171C077F072C0C9
:1030800078F0070E93EC08F0070E93EC08F027C2D7
:103090006BF028C26CF029C26DF02AC26EF0D8EC39
:1030A00017F071C03AF172C03BF171C079F072C093
:1030B0007AF0030E93EC08F000010F01C3CFE8FF94
:1030C000E8CF8BF0C4CFE8FFE8CF8CF0080E93EC8C
:1030D00008F02DC26DF02EC26EF02BC26BF02CC228
:1030E0006CF0D8EC17F071C083F072C084F0090E58
:1030F00093EC08F031C26DF032C26EF02FC26BF06B
:1031000030C26CF0D8EC17F071C085F072C086F058
:103110000A0E93EC08F035C26DF036C26EF033C281
:103120006BF034C26CF0D8EC17F071C087F072C04D
:1031300088F00B0E93EC08F039C26DF03AC26EF0D5
:1031400037C26BF038C26CF0D8EC17F071C089F060
:1031500072C08AF00301B5516EEC24F0D8A0B8EF2C
:1031600018F00001E80E7B6F030E7C6FBDEF18F0C6
:103170000001180E7B6FFC0E7C6F000E93EC08F0C4
:103180003BC26BF03CC26CF03DC26DF03EC26EF0D3
:10319000D8EC17F071C07DF072C07EF0010E93EC98
:1031A00008F03FC26BF040C26CF041C26DF042C209
:1031B0006EF0D8EC17F071C07FF072C080F00301A0
:1031C000B7516EEC24F0D8A0EDEF18F00001E80E36
:1031D000816F030E826F07EF19F00301B9516EEC96
:1031E00024F0D8A0FBEF18F00001180E816FFC0E40
:1031F000826F07EF19F00301B8516EEC24F0D8A0EC
:1032000007EF19F00001000E816F000E826F1200AF
:103210000001106A0FBE101E57EC10F00001640E82
:10322000176E000E186E5BEC11F013C011F014C095
:1032300012F013C00FF014C010F00EAE25EF19F00D
:103240000F1E101E0F2AD8B0102A57EC10F00001E4
:103250000A0E176E000E186E5BEC11F00B50E8CFE3
:1032600017F0186A17BE181E5BEC11F011500D5EB6
:1032700012500E5A13500D2614500E221200030144
:10328000AE516EEC24F073C00DF074C00EF0D8A0F7
:1032900055EF19F003011B510001E8CF0FF00301B6
:1032A0001751E8CF0BF05DEF19F003011A5100013F
:1032B000E8CF0FF0640EE8CF0BF008EC19F00DC06A
:1032C00073F00EC074F00301AF516EEC24F075C0C2
:1032D0000DF076C00EF0D8A079EF19F00301265159
:1032E0000001E8CF0FF003012251E8CF0BF081EF8E
:1032F00019F0030125510001E8CF0FF0640EE8CF6B
:103300000BF008EC19F00DC075F00EC076F003015B
:10331000B0516EEC24F077C00DF078C00EF0D8A05C
:103320009DEF19F0030131510001E8CF0FF00301C7
:103330002D51E8CF0BF0A5EF19F00301305100013A
:10334000E8CF0FF0640EE8CF0BF008EC19F00DC0D9
:1033500077F00EC078F012000301AE516EEC24F04D
:10336000D8A0CBEF19F073C00FF074C010F017C3E2
:103370000DF018C30EF00E6A0DBE0E1E57EC10F0C5
:103380000001640E176E000E186E5BEC11F013C096
:1033900073F014C074F00301AF516EEC24F0D8A0A8
:1033A000EAEF19F075C00FF076C010F022C30DF0EF
:1033B00023C30EF00E6A0DBE0E1E57EC10F0000176
:1033C000640E176E000E186E5BEC11F013C075F0F2
:1033D00014C076F00301B0516EEC24F0D8A009EFD0
:1033E0001AF077C00FF078C010F02DC30DF02EC387
:1033F0000EF00E6A0DBE0E1E57EC10F00001640EAA
:10340000176E000E186E5BEC11F013C077F014C04D
:1034100078F012000201B2519BEC01F00301A751B8
:1034200000010F260301A8510001102218C30DF05E
:1034300019C30EF000010E6AFF0E0DBE0E6E57ECA2
:1034400010F00001640E176E186A196A1A6A5BECB4
:1034500011F000010301195100010D6E0E6A0DBE3D
:103460000E1E0D360E360D5013260E50142213501C
:103470007327145074230201B3519BEC01F0030134
:10348000A95100010F260301AA510001102223C3F4
:103490000DF024C30EF000010E6AFF0E0DBE0E6E7D
:1034A00057EC10F00001640E176E186A196A1A6A58
:1034B0005BEC11F000010301245100010D6E0E6A56
:1034C0000DBE0E1E0D360E360D5013260E50142254
:1034D00013507527145076230201B4519BEC01F070
:1034E0000301AB5100010F260301AC510001102272
:1034F0002EC30DF02FC30EF000010E6AFF0E0DBE9D
:103500000E6E57EC10F00001640E176E186A196AFF
:103510001A6A5BEC11F0000103012F5100010D6EDE
:103520000E6A0DBE0E1E0D360E360D5013260E50B1
:10353000142213507727145078230201B5519BECC5
:1035400001F036C30DF037C30EF000010E6AFF0E16
:103550000DBE0E6E57EC10F00001640E176E186A67
:10356000196A1A6A5BEC11F00301010E3763D0EFA0
:103570001AF00001030E0E6E186EE80E0D6E176E37
:1035800079510D5E7A510E5A196A1A6A13C00FF0FA
:1035900014C010F057EC10F05BEC11F0EAEF1AF0E9
:1035A000020E3763EAEF1AF0000179510D6E7A517D
:1035B0000E6E13C00FF014C010F057EC10F00001A5
:1035C000030EE8CF18F0E80EE8CF17F0196A1A6A70
:1035D0005BEC11F000011350792714507A2312008C
:1035E00000010E6A08C40DF00DBE0E6800010A0E3F
:1035F0000F6E000E106E57EC10F01350732714501E
:10360000742300010E6A09C40DF00DBE0E6800019E
:103610000A0E0F6E000E106E57EC10F01350752747
:103620001450762300010E6A0AC40DF00DBE0E6818
:1036300000010A0E0F6E000E106E57EC10F01350C2
:1036400077271450782300010E6A0BC40DF00DBECD
:103650000E6800010A0E0F6E000E106E57EC10F08F
:103660001350792714507A2300010E6A0CC40DF010
:103670000DBE0E6800010A0E0F6E000E106E57ECA4
:1036800010F013507B2714507C2300010E6A0DC4E8
:103690000DF00DBE0E6800010A0E0F6E000E106ECA
:1036A00057EC10F013507D2714507E2300010E6A52
:1036B0000EC40DF00DBE0E6800010A0E0F6E000E56
:1036C000106E57EC10F013507F2714508023000128
:1036D0000E6A0FC40DF00DBE0E6800010A0E0F6ECB
:1036E000000E106E57EC10F01350812714508223F7
:1036F000120000010A0E0D6E000E0E6E0301BB518A
:103700006EEC24F0D8A0C1EF1BF003014DAF94EF95
:103710001BF04CC30FF0106A0FBE106857EC10F08E
:1037200013C073F014C074F003014FAFA3EF1BF08C
:103730004EC30FF0106A0FBE106857EC10F013C0A4
:1037400075F014C076F0030151AFB2EF1BF050C317
:103750000FF0106A0FBE106857EC10F013C077F02E
:1037600014C078F0030153AFC1EF1BF052C30FF048
:10377000106A0FBE106857EC10F013C079F014C037
:103780007AF00301BC516EEC24F0D8A004EF1CF0D9
:10379000030155AFD7EF1BF054C30FF0106A0FBEF3
:1037A000106857EC10F013C073F014C074F00301EC
:1037B00057AFE6EF1BF056C30FF0106A0FBE10684C
:1037C00057EC10F013C075F014C076F0030159AF38
:1037D000F5EF1BF058C30FF0106A0FBE106857ECDE
:1037E00010F013C077F014C078F003015BAF04EF62
:1037F0001CF05AC30FF0106A0FBE106857EC10F09F
:1038000013C079F014C07AF000017AAF1200E86AB0
:10381000796F7A6F12000201A1B112000301B65153
:103820006EEC24F0D8A012000001606712000201C3
:103830009F510001606F0201010EB66329EF1CF079
:10384000010E00015D6E050E37EC0AF0280E000136
:10385000606F73C00DF074C00EF0CCEC1CF0D8A4F7
:103860005FEF1CF00201B66738EF1CF002019E51B9
:10387000000174BF46EF1CF00301192719AF50EF88
:103880001CF0D8A650EF1CF053EF1CF00301195F99
:1038900019BF50EF1CF0D8A650EF1CF058EF1CF0E9
:1038A00019BF58EF1CF0640E1961196F5DEF1CF021
:1038B000640EE81EE82A1965196F72EC1FF075C0D6
:1038C0000DF076C00EF0CCEC1CF0D8A495EF1CF0F7
:1038D0000201B6676EEF1CF002019E51000176BF37
:1038E0007CEF1CF00301242724AF86EF1CF0D8A640
:1038F00086EF1CF089EF1CF00301245F24BF86EFE4
:103900001CF0D8A686EF1CF08EEF1CF024BF8EEFC3
:103910001CF0640E2461246F93EF1CF0640EE81E0B
:10392000E82A2465246F72EC1FF077C00DF078C090
:103930000EF0CCEC1CF0D8A4CBEF1CF00201B66763
:10394000A4EF1CF002019E51000178BFB2EF1CF001
:1039500003012F272FAFBCEF1CF0D8A6BCEF1CF043
:10396000BFEF1CF003012F5F2FBFBCEF1CF0D8A6E8
:10397000BCEF1CF0C4EF1CF02FBFC4EF1CF0640EB2
:103980002F612F6FC9EF1CF0640EE81EE82A2F6527
:103990002F6F72EC1FF0120000010EAED5EF1CF07D
:1039A0000D1E0E1E0D2AD8B00E2AD8900E320D32E2
:1039B0000E66DFEF1CF0640E0D64E4EF1CF00001F6
:1039C000640E0D6E000E0E6E0D50E832E8321F0BC5
:1039D000D8740DC0E8FF12000001BD6B000174BF78
:1039E000FEEF1CF011C30DF012C30EF073C00FF008
:1039F00074C010F057EC10F008EF1DF015C30DF077
:103A000016C30EF073C00FF074C010F057EC10F036
:103A100013C30DF014C30EF0000114500D26155001
:103A20000E2252EC1EF00DC03CF00EC03DF0000125
:103A300076BF27EF1DF01CC30DF01DC30EF075C03F
:103A40000FF076C010F057EC10F031EF1DF020C3EE
:103A50000DF021C30EF075C00FF076C010F057ECDA
:103A600010F01EC30DF01FC30EF0000114500D2600
:103A700015500E2252EC1EF00DC03AF00EC03BF075
:103A8000000178BF50EF1DF027C30DF028C30EF0E2
:103A900077C00FF078C010F057EC10F05AEF1DF01F
:103AA0002BC30DF02CC30EF077C00FF078C010F0D0
:103AB00057EC10F029C30DF02AC30EF0000114508A
:103AC0000D2615500E2252EC1EF00DC03EF00EC019
:103AD0003FF032C30DF033C30EF079C00FF07AC05F
:103AE00010F057EC10F034C30DF035C30EF00001A8
:103AF00014500D2615500E2252EC1EF00DC040F051
:103B00000EC041F03AC30DF03BC30EF07BC00FF086
:103B10007CC010F057EC10F03CC30DF03DC30EF02C
:103B2000000114500D2615500E2252EC1EF00DC04F
:103B300042F00EC043F0C2EF1DF000017EBFADEFBA
:103B40001DF01CC30DF01DC30EF07DC00FF07EC034
:103B500010F057EC10F0B7EF1DF020C30DF021C3AB
:103B60000EF07DC00FF07EC010F057EC10F01EC3B9
:103B70000DF01FC30EF0000114500D2615500E223B
:103B8000D5EF1DF03EC30DF03FC30EF07DC00FF02A
:103B90007EC010F057EC10F040C30DF041C30EF0A2
:103BA000000114500D2615500E2252EC1EF00DC0CF
:103BB00044F00EC045F002EF1EF0000180BFEDEFB3
:103BC0001DF011C30DF012C30EF07FC00FF080C0C6
:103BD00010F057EC10F0F7EF1DF015C30DF016C301
:103BE0000EF07FC00FF080C010F057EC10F013C340
:103BF0000DF014C30EF0000114500D2615500E22C6
:103C000015EF1EF042C30DF043C30EF07FC00FF05E
:103C100080C010F057EC10F044C30DF045C30EF017
:103C2000000114500D2615500E2252EC1EF00DC04E
:103C300046F00EC047F081C00DF082C00EF00EBEFF
:103C40002AEF1EF046C30FF047C310F057EC10F0F8
:103C500030EF1EF04AC30FF04BC310F057EC10F0DA
:103C600048C30DF049C30EF00D5014260E50152216
:103C700014C00DF015C00EF052EC1EF00DC048F04F
:103C80000EC049F00001CC6751EF1EF00301B151A5
:103C90006EEC24F0D8A051EF1EF038C340F039C3C9
:103CA00041F012000201AE5100010D5C0201AF5162
:103CB00000010E58E8AE62EF1EF0AEC20DF0AFC2CA
:103CC0000EF012000201B05100010D5C0201B15171
:103CD00000010E58E8BE1200B0C20DF0B1C20EF0E5
:103CE0001200000133B480EF1EF035A480EF1EF007
:103CF0003594010E5D6E050E37EC0AF0D880120087
:103D0000D89012000001000E0D6E020E0E6E000122
:103D1000000E136E000E146E010E156EE86A0A6E28
:103D200010EC0CF0020100510001A56F120000011F
:103D3000000E0D6E020E0E6E0001000E136E000ED0
:103D4000146E010E156E040E0A6E44EC0CF0120097
:103D5000E846E8060B6E0001000E0D6E030E0E6EB7
:103D60000001000E136E000E146E010E156E0B5046
:103D70001426E86A1522100E0A6E10EC0CF01200E0
:103D8000E846E8060B6E0001000E0D6E080E0E6E82
:103D90000001000E136E000E146E010E156E0B5016
:103DA0001426E86A1522400E0A6E10EC0CF0000191
:103DB000000EB56F030EB66F0001000EB36F030E59
:103DC000B46F0001080EB46F100EB76F46EC23F00D
:103DD0000001000E0D6E080E0E6E0001000E136E37
:103DE000000E146E010E156E0B501426E86A152293
:103DF000010E0A6E44EC0CF01200E846E8060B6E69
:103E00000001000E0D6E030E0E6E0001000E136E0B
:103E1000000E146E010E156E0B501426E86A152262
:103E20000A6E10EC0CF00001000E0D6E040E0E6E0A
:103E30000001000E136E000E146E010E156E0B5075
:103E4000E82A1426E86A15220A6E10EC0CF012001B
:103E5000E846E8060C6E0001000E0D6E030E0E6EB5
:103E60000001000E136E000E146E010E156E0C5044
:103E70001426E86A1522040E0A6E44EC0CF00001C8
:103E8000000E0D6E040E0E6E0001000E136E000E7D
:103E9000146E010E156E0C50E82A1426E86A1522DD
:103EA000040E0A6E44EC0CF012000001000EB56F17
:103EB000030EB66F0001000EB36F060EB46F000E56
:103EC000B76F46EC23F00001000EB56F040EB66F1D
:103ED0000001000EB36F070EB46F000EB76F46EC13
:103EE00023F0120002010051E846E8060A6E0001C4
:103EF000000E0D6E030E0E6E0001000E136E000E0E
:103F0000146E010E156E0A501426E86A1522010E71
:103F10000A6E44EC0CF0120073C08DF074C08EF089
:103F200075C08FF076C090F077C091F078C092F0B5
:103F300079C093F07AC094F07BC095F07CC096F085
:103F40007DC097F07EC098F07FC099F080C09AF055
:103F500081C09BF082C09CF012008CEC1FF003012A
:103F6000B2516EEC24F0D8B0C8EF1FF0030EE26E31
:103F70005C0EE16E66EC22F0610EE16E66EC22F002
:103F8000660EE16E66EC22F06B0EE16E66EC22F0DE
:103F90008CEC1FF00301B3516EEC24F0D8B0E9EFC4
:103FA0001FF0030EE26E700EE16E66EC22F08CECF8
:103FB0001FF0750EE16E66EC22F08CEC1FF07A0EAD
:103FC000E16E66EC22F08CEC1FF07F0EE16E66EC89
:103FD00022F08CEC1FF00301B4516EEC24F0D8B049
:103FE00004EF20F0030EE26E840EE16E66EC22F028
:103FF000890EE16E66EC22F08E0EE16E66EC22F028
:10400000930EE16E66EC22F012008DC00DF08EC0B2
:104010000EF010C40FF000010EBE11C40FF0106AB4
:104020000FBE106857EC10F00001640E176E000E02
:10403000186E5BEC11F0000113C0E8FF912714C06B
:10404000E8FF922391C00DF092C00EF012C40FF061
:1040500000010EBE13C40FF0106A0FBE106857ECBB
:1040600010F00001640E176E000E186E5BEC11F07C
:10407000000113C0E8FF8D2714C0E8FF8E2391C014
:104080000DF092C00EF014C40FF000010EBE15C466
:104090000FF0106A0FBE106857EC10F00001640EAC
:1040A000176E000E186E5BEC11F0000113C0E8FFF4
:1040B0008F2714C0E8FF902393C00DF094C00EF03A
:1040C00016C40FF000010EBE106A0FBE106857EC48
:1040D00010F00001640E176E000E186E5BEC11F00C
:1040E000000113C0E8FF8F2714C0E8FF90238DC0A4
:1040F00073F08EC074F08FC075F090C076F091C0F0
:1041000077F092C078F093C079F094C07AF004010F
:1041100017A199EF20F08FC07DF090C07EF00401D0
:1041200018A199EF20F000017D1F7E1F7D2BD8B0D4
:104130007E2B030198A1B6EF20F08FC00DF090C048
:104140000EF091C00FF092C010F000010DC075F09C
:104150000EC076F00DC077F00EC078F00F507727C4
:10416000105078230F50755F1050765B030199A1B2
:10417000D3EF20F08FC00DF090C00EF08DC00FF087
:104180008EC010F000010DC075F00EC076F00DC0AD
:1041900073F00EC074F00F507327105074230F503B
:1041A000755F1050765B03019AA18EEF21F08DC0F0
:1041B0000DF08EC00EF00DC073F00EC074F00DC087
:1041C0007FF00EC080F00001640E176E000E186EB6
:1041D00003019C51E812D8B437EF21F0E8BE15EF87
:1041E00021F0640800010F6E106A74BF06EF21F021
:1041F00073C00DF074C00EF057EC10F05BEC11F0D2
:1042000013C073F014C074F037EF21F000017FC0C9
:104210000DF080C00EF057EC10F05BEC11F013C005
:104220007FF014C080F037EF21F0640F00010F6EB3
:10423000106A74AF2AEF21F073C00DF074C00EF055
:1042400057EC10F05BEC11F013C073F014C074F075
:1042500037EF21F000017FC00DF080C00EF057EC69
:1042600010F05BEC11F013C07FF014C080F003017C
:104270009BA141EF21F000017F1F801F7F2BD8B051
:10428000802B0001640E176E000E186E03019D5105
:10429000E812D8B48EEF21F00301C651E812D8B469
:1042A00064EF21F00301C5516EEC24F0D8B08EEF1D
:1042B00021F00001E80E0D6E030E0E6E93510D5E9F
:1042C00094510E5A70EF21F00001E80E0D6E030EAE
:1042D0000E6E99510D269A510E22D8900E320D3243
:1042E0009DC30FF09EC310F0106A0FBE101E57EC56
:1042F00010F05BEC11F0135073271450742303017A
:104300009BB189EF21F00001131E141E132AD8B0AF
:10431000142A000113507F27145080231200030138
:10432000A4A112008CEC1FF005EC20F01200030198
:10433000A4B19FEF21F08CEC1FF005EC20F00301FD
:104340009EA1BAEF21F00301C2516EEC24F0D8A077
:10435000BAEF21F003019F5100010D6E0E6A0001BA
:104360000A0E0F6E000E106E57EC10F013C079F0AD
:1043700014C07AF00301A0A1E7EF21F00301C351BB
:104380006EEC24F0D8A0C9EF21F00301A151D2EFC7
:1043900021F00301C4516EEC24F0D8A0E7EF21F026
:1043A0000301A25100010D6E0E6A00010A0E0F6E8C
:1043B000000E106E57EC10F01350795D14507A59BE
:1043C000E8AEE7EF21F013C079F014C07AF01200E4
:1043D0000BC0E8FFF00BD8B412000DC069F00EC09E
:1043E0006AF00EAEF9EF21F00D1E0E1E0D2AD8B0A8
:1043F0000E2A0DC013F00EC014F0640E176E8AEC76
:1044000010F000011C6A090E136011EF22F00BC0BE
:10441000E8FFE83AE8060F0BE8B62EEF22F023EFAC
:1044200022F0136E0DC01BF00EC01CF0840E0001B4
:104430001B5E030E1C5A0BC0E8FFE83AE8060F0BA0
:10444000E8B62EEF22F00B0DF350460F1324E8CF01
:10445000D9FF020EE8CFDAFF38EF22F0E8960B0D15
:10446000F350DA0F1324E8CFD9FF030EE8CFDAFFB9
:10447000DECF0AF0DFCF0BF000010BC00DF00AC059
:10448000E8FF0D5E0E6A0DBE0E681BC00FF01CC06B
:1044900010F057EC10F00A0E176E8AEC10F00AC0FC
:1044A000E8FF0A0DF3CFE8FF1326F4CFE8FF14224C
:1044B00013C00DF014C00EF000016AAF120000012D
:1044C0000D1E0E1E0D2AD8B00E2A1200E650E8CF9F
:1044D0000BF0E812D8B4120080EC02F0E8EC21F006
:1044E0000DC011F00EC012F0E6CF0AF0E6CFE8FFE3
:1044F0000001E8CF0DF00E6A0DBE0E1E00010A0E7F
:104500000F6E000E106E57EC10F011C00DF012C0BF
:104510000EF013500D5E14500E5A0EBEC5EF22F071
:10452000E6CFE8FF00010AACAEEF22F0E8CF13F0CF
:10453000E9CF14F00DC011F00EC012F0135080EC52
:1045400002F00DC013F00EC014F00A0E176E8AECC4
:1045500010F011C00DF012C00EF013500F6E106A63
:104560000FBE101E57EC10F00001640E176E000E07
:10457000186E196A1A6A5BEC11F013C00DF014C0C2
:104580000EF00A5000EC03F01200E6CFE8FFE6CF91
:10459000E8FF00010AAAE3EF22F0E8CF13F00DC014
:1045A00011F00EC012F0135080EC02F00DC013F0A9
:1045B0000EC014F00A0E176E8AEC10F011C00DF048
:1045C00012C00EF013500F6E106A0FBE101E57EC83
:1045D00010F00001640E176E000E186E196A1A6A48
:1045E0005BEC11F013C00DF014C00EF00A5000EC9B
:1045F00003F012000001BD0EB56F030EB66F00018F
:10460000120EB36F010EB46F050EB76F46EC23F0B8
:10461000D90EE8CFD9FF060EE8CFDAFF060EE8CFB5
:104620000CF0DDCFE8FFE812D8B41EEF23F0DFCFA7
:10463000E8FF6EEC24F0D8B02AEF23F0DDCFE8FFDE
:104640000C2E11EF23F0A5C0E8FF0201006333EF49
:1046500023F01200DECFE8FFDECFE8FF02010063A7
:1046600033EF23F01200E8CF00F2FDEC1EF0000162
:10467000120EB56F010EB66F0001BD0EB36F030EC3
:10468000B46F050EB76F46EC23F012000001B55170
:10469000E16EB651E26E0001B351D96EB451DA6EDB
:1046A000E6CFE8FFE8CFDEFF0001B72F50EF23F0A1
:1046B00012000001BF6B0301AE516EEC24F000014B
:1046C000D8B0BF810301AF516EEC24F00001D8B027
:1046D000BF830301B0516EEC24F00001D8B0BF8558
:1046E0000301B1516EEC24F00001D8B0BF87030183
:1046F000B6516EEC24F00001D8B0BF890301BB5164
:104700006EEC24F00001D8B0BF8B0301BC516EECFD
:1047100024F00001D8B0BF8D1200C00E0FEC0DF0D8
:104720000301AE516EEC24F00001E86AE880BF1589
:10473000D8A0A9EF23F0D8A4BAEF23F0BF71000EE0
:10474000F86E660EF76E7C0EF66E75EC0DF06BEF84
:1047500024F0D8B0BAEF23F0D8B4BAEF23F0BF7189
:10476000000EF86E660EF76E6A0EF66E75EC0DF0C2
:104770006BEF24F00301AF516EEC24F00001E86A06
:10478000E882BF15D8A0D3EF23F0D8A4E4EF23F03C
:10479000BF73000EF86E660EF76EA00EF66E75EC27
:1047A0000DF06BEF24F0D8B0E4EF23F0D8B4E4EFD1
:1047B00023F0BF73000EF86E660EF76E8E0EF66E67
:1047C00075EC0DF06BEF24F00301B0516EEC24F0AA
:1047D0000001E86AE884BF15D8A0FDEF23F0D8A453
:1047E0000EEF24F0BF75000EF86E660EF76EC40E65
:1047F000F66E75EC0DF06BEF24F0D8B00EEF24F0F0
:10480000D8B40EEF24F0BF75000EF86E660EF76E8A
:10481000B20EF66E75EC0DF06BEF24F00301B151A2
:104820006EEC24F00001D8A024EF24F0BFB725EFF0
:1048300024F0BF77000EF86E670EF76E0C0EF66E62
:1048400075EC0DF06BEF24F0BF970301B6516EECE1
:1048500024F00001D8A03BEF24F0BFB93CEF24F0D6
:10486000BF79000EF86E660EF76EFA0EF66E75ECF6
:104870000DF06BEF24F0BF990301BB516EEC24F0F7
:104880000001D8A052EF24F0BFBB53EF24F0BF7B50
:10489000000EF86E660EF76ED60EF66E75EC0DF025
:1048A0006BEF24F0BF9B0301BC516EEC24F00001C0
:1048B000D8A069EF24F0BFBD6AEF24F0BF7D000EE1
:1048C000F86E660EF76EE80EF66E75EC0DF06BEF97
:1048D00024F0BF9D1200500EA36F1200E8AA9AEFB9
:1048E00024F0E8A89AEF24F00A6E070BC90FE16ED6
:1048F000030EE26EE65000010D6E0E6AE8BE0E6811
:1049000000010A0E0F6E000E106E57EC10F00A50E8
:10491000070BE846340FE16E010EE252E650E6CF97
:104920000BF00001135E0B501458E8360ABE12005B
:10493000D8701200D890E8BA1200D880E8B81200F7
:1049400000011F6E206AE8BC2080070BE82AD8808F
:104950002036E82EA8EF24F030501FB63350201434
:10496000D8802062D8901FBED8701200040ED56E79
:104970001200D59E1200D89087B21200D880D5BE02
:104980001200C3C00DF0C4C00EF000013C0E0F6E4B
:10499000000E106E68EC10F013C00DF014C00EF095
:1049A0000001240E0F6EF40E106E68EC10F0C1C002
:1049B00017F0C2C018F00001000E196E000E1A6E3A
:1049C0003EEC13F0A5C317F0A6C318F00001186A57
:1049D0005BEC11F0C00E0FEC0DF0000EF86E650EE2
:1049E000F76EDA0EF66E75EC0DF0CB0E0FEC0DF0E7
:1049F000DBEC0DF0A5C313F0A6C314F0146AC00ECF
:104A00000FEC0DF0D7EC0DF00001000EC36F000E9F
:104A1000C46FD88012000001020E3662120000013D
:104A200033A01200FC6A0AEF05F024EC25F0D8A0B0
:104A30001200FC6A97EC1EF000C2E8FF28EC1FF0A1
:104A400055EC1FF00AEF05F0000130B62EEF25F00F
:104A500032A62EEF25F03296D8801200D8901200A0
:104A60000001670E0E6E300E0D6E77EC25F054ECE3
:104A70000DF00001115080EC01F012001EC10DF08C
:104A80001FC10EF054EC0DF012000001EF51D8B42C
:104A90001200E1CF3EF1E2CF3FF1EDEC17F0000163
:104AA000000E736F000E746F0001000E756F000E24
:104AB000766FACEC19F03FEC19F079EC1BF00BECD5
:104AC0001CF00AEC1AF08FEC21F0ADEC1FF097EC23
:104AD00021F0F0EC1AF0ECEC1CF04EEC0EF03EC1C4
:104AE000E1FF3FC1E2FF12000001EF6912000BEC91
:104AF00025F00001CD6BDB6BEA6BEB6BC00E0FECAE
:104B00000DF00DC0F6FF0EC0F7FFF86A0DC00FF0F4
:104B10000EC010F075EC0DF0FA0E9DEC0BF07EEC73
:104B200029F0D8A49AEF25F0110E0D26D8B00E2A40
:104B3000A1EF25F0D8A0AEEF25F0130E0D26D8B0CA
:104B40000E2A0DC0F6FF0EC0F7FFF86A0900F5CF78
:104B50000DF00900F5CF0EF07EEF25F015EC25F0F5
:104B600071EC1EF0D8A07EEF25F0150E0D26D8B002
:104B70000E2A0DC0F6FF0EC0F7FFF86A0900F5CF48
:104B800011F00900F5CF12F00FC00DF010C00EF0BB
:104B90000900F5CF0FF00900F5CF10F00900F5CFAF
:104BA000CEF00900F5CFCFF00001B96BBA6BBB694D
:104BB0007F0EE8CFBCF012ACEAEF25F00900F5CF8C
:104BC000B9F00900F5CFBAF00900F5CFBBF0090044
:104BD000F5CFBCF012A4F3EF25F00900F5CFEAF011
:104BE0000900F5CFEBF012A2FCEF25F00900F5CF9C
:104BF000ECF00900F5CFEDF012AE01EF26F054EC29
:104C00000DF012A606EF26F06AEC0DF012A21200CB
:104C10000001E86AE8CFFBFFEDC0E8FFE8CFFAFF4C
:104C2000ECC0E8FFF96EE8CF0AF00FC01BF010C02F
:104C30001CF00FC0F6FF10C0F7FFF86A150EF6263D
:104C4000D8B0F72A0900F5CFE8FF0A6229EF26F06D
:104C500012000FC0F6FF10C0F7FF110EF626D8B0F5
:104C6000F72A0900F5CF0FF00900F5CF10F00FC0BB
:104C7000E8FF1B6219EF26F010C0E8FF1C6219EF75
:104C800026F01200000110500F10D8B41200E86A8C
:104C9000FB6E1050E8CFFAFF0F50F96E00010F5075
:104CA000E16E1050E26E0001000E11626CEF26F012
:104CB0000FC0F6FF10C0F7FFF86A160EF626D8B040
:104CC000F72ACEC0E1FFCFC0E2FFE7CFE8FF13EC49
:104CD00026F0EBEC28F01200010E116273EF26F0C3
:104CE00015EC28F01200020E11629DEF26F0000173
:104CF00012A07EEF26F0CE510001B86FE6CF0AF089
:104D0000E5CF0BF000010AC011F00BC012F0129EAB
:104D1000129C6BEC28F000010FC0E1FF10C0E2FF15
:104D200011C00AF012C00BF00AC0E6FFE7CFE8FF9F
:104D3000C00B0B120BC0E5FF1200030E1162B2EFA5
:104D400026F0E7CFE8FFE8366EEC27F0000ED8B08B
:104D5000E81E0A6E00010FC0E1FF10C0E2FF0AC0AA
:104D6000E7FF1200040E1162C3EF26F0E7CFE8FF61
:104D700032EC29F00A6E00010FC0E1FF10C0E2FF23
:104D80000AC0E7FF1200050E1162D5EF26F0E7CF4B
:104D9000E8FFC3EC27F0E8CF0AF000010FC0E1FF05
:104DA00010C0E2FF0AC0E7FF1200060E1162EBEF2F
:104DB00026F0E7CF0AF00FC0CEF010C0CFF0000110
:104DC000E40E0F6E7A0E106E0AC0E8FF13EC26F0A8
:104DD000EBEC28F01200070E1162F2EF26F042EC25
:104DE00026F01200080E116203EF27F0E7CFE8FF6C
:104DF000BDEC27F0E8CF0AF000010FC0E1FF10C0C2
:104E0000E2FF0AC0E7FF0A0E116224EF27F0E7CFA6
:104E1000E8FF0001CE15D890D8B4D8806EEC27F00A
:104E20000001CEC00AF000010FC0E1FF10C0E2FF98
:104E3000D8B01FEF27F00AC0E8FFE71212000AC03F
:104E4000E8FFE81EE716120012000B6AD8B00B1E2E
:104E5000C00E0FEC0DF0000EF86E650EF76E800EB2
:104E6000F66E75EC0DF00BA04AEF27F0C80E0FECB4
:104E70000DF0280E00EC0DF0CC0E0FEC0DF0290E0D
:104E800000EC0DF0CF0E0FEC0DF0200E00EC0DF04D
:104E90005CEF27F0C80E0FEC0DF0200E00EC0DF0CB
:104EA000CC0E0FEC0DF0280E00EC0DF0CF0E0FEC39
:104EB0000DF0290E00EC0DF07EEC29F0D8B40B6A51
:104EC000FF0ED8B00B6E15EC25F071EC1EF0D8A0DB
:104ED00033EF27F0D8900BB0D88012000B6AD8B00F
:104EE0000B1EC80E0FEC0DF0000EF86E650EF76E7F
:104EF000BE0EF66E75EC0DF00BA093EF27F0C80E0A
:104F00000FEC0DF0280E00EC0DF0CC0E0FEC0DF0B8
:104F1000290E00EC0DF0CF0E0FEC0DF0200E00EC82
:104F20000DF0A5EF27F0C80E0FEC0DF0200E00ECF1
:104F30000DF0CC0E0FEC0DF0280E00EC0DF0CF0EA6
:104F40000FEC0DF0290E00EC0DF07EEC29F0D8B43A
:104F50000B6AFF0ED8B00B6E15EC25F071EC1EF04D
:104F6000D8A07CEF27F0D8900BB0D88012000001B9
:104F7000BB65BB51B961B95112000001E86900017C
:104F80009D6FC7EF27F000019D6F0001E86BC80E11
:104F90009DEC0BF09DC0E8FF0001136E146A156ACA
:104FA000166A05EC0EF00001E867E5EF27F0CD0E7C
:104FB0000FEC0DF0275000EC0DF0285000EC0DF038
:104FC000295000EC0DF0F4EF27F0CC0E0FEC0DF0B3
:104FD000275000EC0DF0285000EC0DF02E0E00ECE8
:104FE0000DF0295000EC0DF0A4EC29F00001D8A43C
:104FF00000EF28F09D2BBB519D619D6F0BEF28F0BA
:10500000D8A00BEF28F09D51B9610BEF28F09D0758
:10501000B9519D659D6F15EC25F071EC1EF0D8A07F
:10502000C7EF27F000019D51120045EC25F0FA0E64
:105030009DEC0BF0E7CFE8FFE7BEE81EE7BEE82AED
:105040000001136E146A156A166A05EC0EF0CB0E99
:105050000FEC0DF0200EE7BE2D0E00EC0DF02750EA
:1050600000EC0DF0285000EC0DF0295000EC0DF094
:10507000250E00EC0DF0A4EC29F00001D8A444EFBB
:1050800028F0E72A48EF28F0D8A048EF28F0E706F4
:1050900015EC25F071EC1EF0D8A015EF28F00001FA
:1050A000EF6B120000011150BB5D1250BC59D8B01B
:1050B0005FEF28F0BB51116EBC51126E1200B95156
:1050C000115CBA511258D8B06AEF28F0B951116E7C
:1050D000BA51126E120052EC28F00001BE6B0001B2
:1050E000B851E812D8B47DEF28F0B851E16E000E47
:1050F000E26E11C0E6FF12C0E7FFF0C0E8FF7F08D4
:10510000E8BEE86AE8669DEC0BF011C013F012C02F
:1051100014F0D89014321332156A166A05EC0EF0AA
:10512000C90E0FEC0DF0265000EC0DF02E0E00EC29
:105130000DF0275000EC0DF0285000EC0DF0295038
:1051400000EC0DF06D0E00EC0DF0530E00EC0DF0C8
:10515000A4EC29F00001D8A4BDEF28F0112AD8B49E
:10516000122A112AD8B4122ABC5112626BEF28F00D
:10517000BB511160116E6BEF28F0D8A0CFEF28F073
:105180001106D8A012061106D8A01206BA51126252
:105190006BEF28F0B9511164116E6BEF28F000012C
:1051A00033A2BE6933BCDAEF28F00001A00E116E05
:1051B0000F0E126E000133BEE3EF28F00001D00E97
:1051C000116E070E126E15EC25F071EC1EF0D8A0D2
:1051D0006FEF28F01200C00E0FEC0DF00FC0F6FFBD
:1051E00010C0F7FF75EC0DF0FA0E9DEC0BF0A4EC7F
:1051F00029F0D8A402EF29F0110E0F26D8B0102AFA
:1052000009EF29F0D8A016EF29F0130E0F26D8B019
:10521000102A0FC0F6FF10C0F7FFF86A0900F5CF9B
:105220000FF00900F5CF10F0EBEF28F015EC25F0AA
:1052300071EC1EF0D8A0EBEF28F0150E0F26D8B0B9
:10524000102A0FC0F6FF10C0F7FFF86A0900F5CF6B
:105250000AF00900F550CEC0E1FFCFC0E2FF0AC05E
:10526000E7FF12000F0BE8B6080B0C0DF3CF13F09D
:10527000F4CF14F00001180E1326710E1422CC0E78
:105280000FEC0DF013C0F6FF14C0F7FF75EC0DF036
:10529000FA0E9DEC0BF0A4EC29F0D8A456EF29F0FF
:1052A000050E1326D8B0142A5DEF29F0D8A06AEFB6
:1052B00029F0070E1326D8B0142A13C0F6FF14C025
:1052C000F7FFF86A0900F5CF13F00900F5CF14F0E5
:1052D0003FEF29F015EC25F071EC1EF0D8A03FEF60
:1052E00029F0090E1326D8B0142A13C0F6FF14C0F3
:1052F000F7FFF86A0900F5CFE8FF1200040E93ECFF
:1053000008F0040E93EC08F0C5C0E8FFC35EC6C009
:10531000E8FFC45AC4BE97EF29F0640EC35E000EC6
:10532000C45AC4BEA1EF29F0D884D8901200640EEC
:10533000C326000EC422C4AEA1EF29F0D894D880B1
:105340001200D894D8901200050E93EC08F0050EC8
:1053500093EC08F0C7C0E8FFC35EC8C0E8FFC45ABA
:10536000C4BEC1EF29F0640EC35E000EC45AC4BEB1
:10537000D1EF29F0C466C368C3CFF0F0D884D890C9
:105380001200640EC326000EC422C4AED1EF29F071
:10539000C31EC41EC466C368C3CFF0F0D894D880BF
:1053A0001200D894D8901200CEEF2AF0800E0FECA5
:1053B0000DF0000EF86E670EF76E480EF66E75EC87
:1053C0000DF01BEF2BF00101600E1E6F670E1F6FBB
:1053D00001014C0E206F690E216F5EEC2AF097ECF4
:1053E0001EF000C2E8FF28EC1FF055EC1FF0120081
:1053F0000101780E1E6F670E1F6F01013E0E206FB8
:105400006A0E216F5EEC2AF0EFEF29F00101900E99
:105410001E6F670E1F6F0101280E206F6C0E216F2B
:105420005EEC2AF0EFEF29F00101A80E1E6F670E67
:105430001F6F0101840E206F710E216F5EEC2AF048
:10544000EFEF29F00101C00E1E6F670E1F6F010103
:10545000520E206F780E216F5EEC2AF0EFEF29F0EC
:105460000001DD6B0101D80E1E6F670E1F6F010179
:105470005C0E206F7E0E216F5EEC2AF0EFEF29F0BC
:105480000101F00E1E6F670E1F6F0101A40E206F49
:10549000820E216F5EEC2AF0EFEF29F00101080E79
:1054A0001E6F680E1F6F01011E0E206F860E216F8A
:1054B0005EEC2AF0EFEF29F0F3EF31F03EEC25F04F
:1054C00020C10DF021C10EF077EC25F00DC020F1C8
:1054D0000EC021F1EAC026F1EBC027F10001115006
:1054E000090AD8A4C0EF2AF00FC00DF010C00EF0CA
:1054F00077EC25F00DC022F10EC023F1EAC028F1AF
:10550000EBC029F100011150090AD8A4A8EF2AF034
:105510000FC00DF010C00EF077EC25F00DC024F197
:105520000EC025F1EAC02AF1EBC02BF14EEC26F0BB
:105530000001CDB1AEEF2AF02AC10FF02BC110F05F
:1055400042EC26F024C10DF025C10EF08CEF2AF0BC
:105550004EEC26F00001CDB1C5EF2AF028C10FF0C6
:1055600029C110F042EC26F020C10DF021C10EF04F
:1055700054EC0DF022C10DF023C10EF078EF2AF0AB
:105580004EEC26F00001CDB1120026C10FF027C16C
:1055900010F042EC26F05EEF2AF0120000C2E8FFA5
:1055A000A8EC1EF0800E0FEC0DF0000EF86E650EEC
:1055B000F76E4A0EF66E75EC0DF08D0E0FEC0DF0D9
:1055C000020100510001136E146A156A166AD3ECC9
:1055D0000DF0CDEC05F0FA0E9DEC0BF0A4EC29F0EB
:1055E000D8A4FDEF2AF0610E0201002B0063CEEF7C
:1055F0002AF0010E006FCEEF2AF0D8A00BEF2BF0AF
:1056000002010007000E0063CEEF2AF0600E0201D7
:10561000006FCEEF2AF071EC1EF0D8A0EEEF2AF06A
:1056200000C2E8FFFDEC1EF000C2E8FFE8CFA5F0E5
:1056300097EC1EF01200C00E0FEC0DF0CDEC05F053
:10564000000EE16E030EE26E960E9DEC0BF0C00EA6
:10565000E1240FEC0DF0E75000EC0DF0C00EE1245A
:105660000FEC0DF00E0E0FEC0DF07EEC29F0D8A42F
:1056700043EF2BF0E12A0F0EE16424EF2BF0000E34
:10568000E16E24EF2BF0D8A04FEF2BF0E106FF0ED8
:10569000E16224EF2BF00F0EE16E24EF2BF0A4EC6F
:1056A00029F0D8A45AEF2BF0E72A7A0EE760E76ECC
:1056B00024EF2BF0D8A063EF2BF0E706200EE76471
:1056C000E76E24EF2BF071EC1EF0D8A035EF2BF035
:1056D0000C0E0FEC0DF000C2E8FF28EC1FF01200DA
:1056E0000DC02CF10EC02DF10FC02EF110C02FF106
:1056F000D0C00DF0D1C00EF00001E80E0F6E030E09
:10570000106E57EC10F00001000E176E010E186EAF
:105710005BEC11F013C0D0F014C0D1F00001D251F5
:10572000D027D351D123D4C00DF0D5C00EF0000145
:10573000E80E0F6E030E106E57EC10F00001000E15
:10574000176E010E186E5BEC11F0D2C0D4F0D3C00E
:10575000D5F01350D45F1450D55BD0C00DF0D1C03C
:105760000EF052EC1EF00DC0D0F00EC0D1F0D2C041
:105770000DF0D3C00EF052EC1EF00DC0D2F00EC0F2
:10578000D3F0D4C00DF0D5C00EF052EC1EF00DC019
:10579000D4F00EC0D5F02CC10DF02DC10EF02EC1ED
:1057A0000FF02FC110F012000DC02CF10EC02DF122
:1057B0000FC02EF110C02FF1D0C00DF0D1C00EF0EF
:1057C0000001E80E0F6E030E106E57EC10F0000192
:1057D000000E176E010E186E5BEC11F0D2C0D0F007
:1057E000D3C0D1F000011350D0271450D12313504F
:1057F000D25F1450D35BD0C00DF0D1C00EF052EC8C
:105800001EF00DC0D0F00EC0D1F0D2C00DF0D3C04C
:105810000EF052EC1EF00DC0D2F00EC0D3F02CC131
:105820000DF02DC10EF02EC10FF02FC110F012009F
:105830000DC02CF10EC02DF10FC02EF110C02FF1B4
:10584000D0C00DF0D1C00EF0D2510D5ED3510E5A22
:105850000001000E0F6E010E106E57EC10F00001EB
:10586000E80E176E030E186E5BEC11F013C0D0F04B
:1058700014C0D1F0D2C00DF0D3C00EF0D4510D5EE3
:10588000D5510E5A0001000E0F6E010E106E57EC2E
:1058900010F00001E80E176E030E186E5BEC11F0AD
:1058A00013C0D4F014C0D5F02CC10DF02DC10EF0F2
:1058B0002EC10FF02FC110F012000DC02CF10EC040
:1058C0002DF10FC02EF110C02FF1D0C00DF0D1C0BE
:1058D0000EF00001D2510D5ED3510E5A0001000EA0
:1058E0000F6E010E106E57EC10F00001D00E176E07
:1058F000070E186E5BEC11F013C0D0F014C0D1F09D
:10590000D0C00DF0D1C00EF00001E80E0F6E030EF6
:10591000106E57EC10F00001000E176E010E186E9D
:105920005BEC11F000011350D2271450D3232CC18B
:105930000DF02DC10EF02EC10FF02FC110F012008E
:105940000DC02CF10EC02DF10FC02EF110C02FF1A3
:105950000001BEA1D8EF2CF0000E00010F18D8B442
:10596000C3EF2CF0D2C013F0D3C014F0D89013368C
:105970001436D051135ED151145A13C0D4F014C050
:10598000D5F0D8EF2CF0000E00010F18D8B4D8EFE6
:105990002CF0D2C013F0D3C014F0D89013361436C4
:1059A000D451135ED551145A13C0D0F014C0D1F0A5
:1059B0002CC10DF02DC10EF02EC10FF02FC110F033
:1059C00012003C0E0001B86F0001110EB56F030EFE
:1059D000B66F0001D00EB36F000EB46F0B0EB76F31
:1059E00046EC23F0DB6B70EC2BF012003A0E00015A
:1059F000B86F00011C0EB56F030EB66FE9EF2CF007
:105A00003E0E0001B86F0001270EB56F030EB66F92
:105A1000E9EF2CF00001110EB36F030EB46FA0EC90
:105A20002CF0DBA1D86B18EC2CF00001D00EB56F78
:105A3000000EB66F0B0EB76F46EC23F00001B86B8B
:105A4000120000011C0EB36F030EB46F0FEF2DF0A8
:105A50000001270EB36F030EB46F0FEF2DF00DC0D2
:105A60002CF10EC02DF10FC02EF110C02FF103014B
:105A700032C30DF033C30EF00001E80E0F6E030EBB
:105A8000106E57EC10F00001000E176E010E186E2C
:105A90005BEC11F013C032F314C033F30301345143
:105AA0003227355133232CC10DF02DC10EF02EC1FC
:105AB0000FF02FC110F012000DC02CF10EC02DF10F
:105AC0000FC02EF110C02FF132C30DF033C30EF012
:105AD0000301345100010D5E0301355100010E5ADE
:105AE0000001000E0F6E010E106E57EC10F0000159
:105AF000E80E176E030E186E5BEC11F013C032F354
:105B000014C033F32CC10DF02DC10EF02EC10FF0D7
:105B10002FC110F00001B86B1200420E0001B86FE7
:105B200000013A0EB56F030EB66F0001D00EB36FD1
:105B3000000EB46F040EB76F46EC23F0D4EC2BF0DC
:105B40001200440E0001B86F00013E0EB56F030E47
:105B5000B66F95EF2DF0460E0001B86F0001420EB2
:105B6000B56F030EB66F95EF2DF000013A0EB36FCF
:105B7000030EB46F5DEC2CF00001D00EB56F000E7B
:105B8000B66F040EB76F46EC23F00001B86B12003D
:105B900000013E0EB36F030EB46FBAEF2DF000019B
:105BA000420EB36F030EB46FBAEF2DF00001460E34
:105BB000B56F030EB66F0001D00EB36F000EB46F59
:105BC000060EB76F46EC23F070EC2BF0120018ECC9
:105BD0002CF00001D00EB56F000EB66F0001460E1E
:105BE000B36F030EB46F060EB76F46EC23F00001DF
:105BF000B86B1200AEC2B9F0AFC2BAF0B0C2BBF01F
:105C0000B1C2BCF01200CEC0B5F0CFC0B6F00001FA
:105C1000DC0EB36F000EB46F050EB76F46EC23F0C9
:105C2000CEC0B3F0CFC0B4F00001DC51E83A0F0BA6
:105C3000E46FE36BDDBFE31FE16BDF51DDBDE16FBF
:105C4000E26BE051DDBBE26F0F0EE117E217DD17EB
:105C5000DC1712000001E451E83AF00BDC13E3BF5B
:105C6000DD8FE151E812D8B439EF2EF0E151DF6F4A
:105C7000DD8DE251E812D8B441EF2EF0E251E06F31
:105C8000DD8B0001DC0EB56F000EB66F050EB76F31
:105C900046EC23F0120010C4DFF011C4E0F0120053
:105CA000DFC010F4E0C011F4120012C4DFF013C41E
:105CB000E0F01200DFC012F4E0C013F4120014C4CC
:105CC000DFF015C4E0F01200DFC014F4E0C015F4FA
:105CD00012000001DBAF12000301196B246B2F6B64
:105CE00012000001DBAF1200A7C313F0A8C314F029
:105CF000835113268451142213C0A7F314C0A8F3B0
:105D0000A9C313F0AAC314F0855113268651142297
:105D100013C0A9F314C0AAF3ABC313F0ACC314F0BF
:105D2000875113268851142213C0ABF314C0ACF36F
:105D300012000001DBAF12000301A76BA86BA96B77
:105D4000AA6BAB6BAC6B12000001B96BB92B600E88
:105D50000001BB6F12000001DD51DD67B1EF2EF0D5
:105D60001200020100C20AF0006F00010AC0DDF05B
:105D700028EC1FF00001DDC00AF002010AC000F2A9
:105D800012000001DBAF120003011951196B18C397
:105D90000AF000010D6E0E6AE8BE0E680D360E3672
:105DA0000001640E0F6E000E106E57EC10F00AC06A
:105DB00017F0186A5BEC11F013500301A7270001DC
:105DC00014500301A82303012451246B23C30AF0B8
:105DD00000010D6E0E6AE8BE0E680D360E3600012B
:105DE000640E0F6E000E106E57EC10F00AC017F024
:105DF000186A5BEC11F013500301A927000114503D
:105E00000301AA2303012F512F6B2EC30AF00001B7
:105E10000D6E0E6AE8BE0E680D360E360001640E79
:105E20000F6E000E106E57EC10F00AC017F0186AD3
:105E30005BEC11F013500301AB2700011450030178
:105E4000AC2312000001DBAF120054EC32F0120060
:105E500046EC23F012000001D00EB36F000EB46FB9
:105E6000CEC0B5F0CFC0B6F00B0EB76F46EC23F046
:105E70000001D00EB56F000EB66FCEC0B3F0CFC02C
:105E8000B4F00B0EB76F12000201D890A2371200C7
:105E90000201D890A23312000001E9AF120001EC18
:105EA00010F0120013C20FF014C210F0030E000124
:105EB000A06F03EC31F00FC013F210C014F2120007
:105EC000A9C20FF0AAC210F00D0E0001A06F03ECE2
:105ED00031F00FC0A9F210C0AAF212000001DBAF2E
:105EE00012000501006B016B0201B8691200C9ECD8
:105EF0000BF012000001CE51B36F020EB46FCF5100
:105F000000011F6E030E7EEC08F014C08BF015C06C
:105F10008CF0C00E0FEC0DF0000EF86E8C0EF76ECC
:105F2000360EF66E75EC0DF071EC1EF0D8A094EF05
:105F30002FF000011F507EEC08F014C06DF015C06A
:105F40006EF014C06FF015C070F0FA0E9DEC0BF0FF
:105F5000C00E0FEC0DF0000EF86E8C0EF76E480EB2
:105F6000F66E75EC0DF071EC1EF0D8A0B3EF2FF0CB
:105F700000011F507EEC08F014C06BF015C06CF0EF
:105F8000FA0E9DEC0BF000016B516D276C516E23E6
:105F90006E336D336E9F6FC017F070C018F0000144
:105FA000E80E146E030E156E136A166A6B51175EB7
:105FB0006C51185A18321732187E196A1A6A5BEC3B
:105FC00011F013C06BF014C06CF000016B0EB56FD4
:105FD000000EB66F040E0001B76F46EC23F01200FE
:105FE0000001CE51B36F020EB46FCF5100011F6E8E
:105FF000C00E0FEC0DF0000EF86E8C0EF76E360E24
:10600000F66E75EC0DF071EC1EF0D8A003EF30F0D9
:1060100000011F507EEC08F014C06BF015C06CF04E
:10602000FA0E9DEC0BF0C00E0FEC0DF0000EF86EAA
:106030008C0EF76E480EF66E75EC0DF071EC1EF0DE
:10604000D8A01EEF30F000011F507EEC08F014C005
:106050006DF015C06EF0FA0E9DEC0BF00001E80E2D
:10606000146E030E156E136A166A6BC017F06CC0BF
:1060700018F0196A1A6A00016D51175E6E51185AAC
:1060800018AE44EF30F0FF0E196E1A6E5BEC11F093
:1060900013C06BF014C06CF000016B0EB56F000EF6
:1060A000B66F040E0001B76F46EC23F0120000013A
:1060B000CE51B36F020EB46FCF5100011F6EC00EF0
:1060C0000FEC0DF0000EF86E8C0EF76E240EF66ECF
:1060D00075EC0DF071EC1EF0D8A06AEF30F0000105
:1060E0001F507EEC08F0000113361436153614C02C
:1060F0006DF015C06EF0FA0E9DEC0BF0C00E0FECBB
:106100000DF0000EF86E8C0EF76E360EF66E75EC16
:106110000DF071EC1EF0D8A089EF30F000011F5097
:106120007EEC08F0000113361436153614C06BF0FF
:1061300015C06CF0FA0E9DEC0BF0C00E0FEC0DF0DC
:10614000000EF86E8C0EF76E480EF66E75EC0DF0C4
:1061500071EC1EF0D8A0A8EF30F000011F507EECCB
:1061600008F0000113361436153614C06FF015C050
:1061700070F0FA0E9DEC0BF00001E80E146E030EA9
:10618000156E136A166A6BC017F06CC018F0196AA6
:106190001A6A00016D51175E6E51185A18AED2EF8F
:1061A00030F0FF0E196E1A6E5BEC11F013C06BF03D
:1061B00014C06CF00001E80E146E030E156E136A25
:1061C000166A6DC017F06EC018F0196A1A6A0001DD
:1061D0006F51175E7051185A18AEF0EF30F0FF0E85
:1061E000196E1A6E5BEC11F013C06FF014C070F0F2
:1061F00000016B0EB56F000EB66F060E0001B76F93
:1062000046EC23F01200140E9DEC0BF00001A0519F
:1062100093EC08F0C00E0FEC0DF0000EF86E680E57
:10622000F76EE00EF66E75EC0DF0CB0E0FEC0DF088
:1062300069C00DF06AC00EF057EC10F01450136EE8
:106240001550146E156A05EC0EF0200E0A6E300E15
:1062500025640AC025F0255000EC0DF0265000EC16
:106260000DF02E0E00EC0DF0275000EC0DF0285034
:1062700000EC0DF0A4EC29F0D8A445EF31F00001BA
:106280000F2AD8B4102A03EF31F0D8A04FEF31F025
:1062900000010F06FF0E0F60100603EF31F071ECE6
:1062A0001EF0D8A003EF31F012000201FF0EA5632B
:1062B00067EF31F000019D510FEC0DF0000EF86E0C
:1062C000650EF76E6E0EF66E75EC0DF012000201A3
:1062D000D1B185EF31F0D1A385EF31F000019D51AF
:1062E0000FEC0DF0000EF86E650EF76E5C0EF66E9C
:1062F00075EC0DF000019D51080F0FEC0DF002013F
:10630000310EA52500EC0DF012000201D1A1BAEF6B
:1063100031F0D1B3BAEF31F000019D510FEC0DF027
:10632000000EF86E650EF76EC80EF66E75EC0DF089
:1063300000019D510E0F0FEC0DF00201300EA5254E
:1063400000EC0DF00201A551D890E836500F000185
:10635000136E146A156A166A05EC0EF000019D5161
:10636000040F0FEC0DF0285000EC0DF0295000EC5C
:106370000DF012000201D1A11200D1A31200000100
:106380009D510FEC0DF0000EF86E660EF76E340E98
:10639000F66E75EC0DF000019D510D0F0FEC0DF038
:1063A0000201A55101010E250001136E146A156A40
:1063B000166AD3EC0DF00201A551D890E836010F12
:1063C0000001136E146A156A166A05EC0EF00001DE
:1063D0009D51040F0FEC0DF0285000EC0DF02950EA
:1063E00000EC0DF012000301FF0EAD6308EF32F078
:1063F000C00E0FEC0DF0000EF86E650EF76E6E0E0F
:10640000F66E75EC0DF0FA0E9DEC0BF014EF32F019
:106410000301AD510201A56FC00E00019D6F55EC47
:1064200031F0FA0E9DEC0BF0A4EC29F0D8A424EF87
:1064300032F0010110510301AD2BAD63F3EF31F0E8
:10644000FF0EAD6FF3EF31F0D8A034EF32F003015F
:10645000AD07FE0EAD63F3EF31F001011051E80618
:106460000301AD6FF3EF31F071EC1EF0D8A014EF23
:1064700032F000C2E8FF28EC1FF01200000EF86EA8
:106480008C0EF76E5A0EF66E000E0A6E020EE26E5B
:10649000000EE16E0900F550E66E0A060900F5509F
:1064A000E66E0A2E4AEF32F0000EF86E8D0EF76E91
:1064B0005A0EF66E000E0A6E030EE26E000EE16ECC
:1064C0000900F550E66E0A060900F550E66E0A2E40
:1064D00060EF32F0000EF86E8E0EF76E5A0EF66E0A
:1064E000000E0A6E040EE26E000EE16E0900F55019
:1064F000E66E0A060900F550E66E0A2E76EF32F0D7
:1065000012002020202020202020202020202020B9
:1065100020200000204D6963726F53746172203235
:10652000303030200000202056657273696F6E2075
:10653000322E30652020000041444320434820583B
:1065400058203D205858585800002020204169729A
:106550006372616674202320202000002020202008
:106560002035332E58204D487A202020000020204E
:1065700020202020204F46462020202020200000E0
:10658000204163636570743F20596573204E6F200E
:1065900000002050726573732020204F7074696F63
:1065A0006E200000202020202020200020202020FD
:1065B00053747564656E74202020202000002059DB
:1065C0006573204E6F2000002035302E5858204D26
:1065D000487A202043485820000078426C642052BA
:1065E000504D203D2078787878780000526574729C
:1065F0006163747320617265205550210000202072
:10660000466F726D617420466C61736820200000D3
:106610002020466F726D6174696E672E2E2E2020C9
:106620000000202020436F7079696E672E2E2E2087
:10663000202000002037322E5858204D487A204321
:1066400048585820000052454320566F6C74733DE3
:106650002058582E585800005468726F74746C6536
:10666000202041646A7573740000202041494C2049
:10667000442F52204849474820200000202041490B
:106680004C20442F5220204C4F5720200000202027
:10669000454C4520442F52204849474820200000BF
:1066A0002020454C4520442F5220204C4F5720207D
:1066B0000000202052554420442F5220484947488A
:1066C00020200000202052554420442F5220204CEE
:1066D0004F5720200000202020534E415020524987
:1066E0004748542020200000202020534E415020B5
:1066F000204C4546542020200000202020415554A5
:106700004F20205452494D202020000020202020DE
:1067100020505245534554202020202000002020A6
:106720002043414C49425241544520202020000042
:1067300053656C656374202041697263726166748D
:106740000048673868000000204169726372616622
:106750007420206E616D6520006067306704000062
:1067600020202020202054696D65722020202020C8
:106770000078674867080000202020202020536E02
:10678000617020202020202000906760670C0000AE
:106790002020202020536572766F73202020202037
:1067A00000A867786710000020202020204D69781D
:1067B000657273202020202000C0679067140000BD
:1067C0002020202020537769746368202020202017
:1067D00000D867A867180000202020204F70746937
:1067E0006F6E73202020202000F067C0671C00001F
:1067F00020536861726564204F7074696F6E7320F6
:10680000000868D867200000202053797374656DF4
:106810002053657475702020002068F06724000004
:1068200053656C656374204672657175656E637936
:1068300000386808682800002020202020204558C3
:10684000495420202020202000306720682C0000A0
:10685000456E61626C6520202020202020202020B1
:1068600000005265736574203F20202020202020E6
:10687000202000005A65726F20203F202020202019
:10688000202020200000436C656172203F202020E2
:10689000202020202020000041697263726166740C
:1068A00020232020202020200000546F2041465427
:1068B000202320202020202020200000426C616422
:1068C0006573203D202020202020202000004678D5
:1068D0006420467273742020202020202020000095
:1068E000566F6C7473202020202020202020202030
:1068F0000000576964746820202020202020202078
:10690000202000004368616E6E656C73202020209B
:106910002020202000004E656753686966743F2080
:106920002020202020200000506F73203D202020B8
:10693000202020202020202000004761696E202098
:106940002020202020202020202000002020202087
:1069500020204D6F6465202020202020006869DC05
:10696000690080F669BD03004D696E75746573201A
:1069700020202020202020200088694C690540BF6D
:106980000300000000FF00005365636F6E64732016
:10699000202020202020202000A86968690540BE12
:1069A0000300000000FF000020456E61626C65205E
:1069B000205377697463682000C26988690680C0C3
:1069C00003005468726F74746C65202020202020AE
:1069D000202000DC69A8690100C103004558495422
:1069E000202020202020202020202020004C69C2B0
:1069F000690300CD00002020202055502054696DEF
:106A0000657220202020000E6A266A0000002020E7
:106A100020446F776E2054696D6572202020002617
:106A20006AF669010000446F776E202053746F701E
:106A30002054696D657200F6690E6A0200005352B7
:106A40002041494C20202020202020202020005EB2
:106A50006A0E6C01404C030000FF007E00005352A0
:106A600020454C4520202020202020202020007E72
:106A70006A3E6A01404E030000FF007E0000535250
:106A80002052554420202020202020202020009E1D
:106A90006A5E6A014050030000FF007E000053520E
:106AA000205448542020202020202020202000BED8
:106AB0006A7E6A014052030000FF007E00005352CC
:106AC0002041494C203F202020202020202000D899
:106AD0006A9E6A03004D0300535220454C45203FF7
:106AE000202020202020202000F26ABE6A03004FD0
:106AF0000300535220525544203F202020202020C4
:106B00002020000C6BD86A0300510300535220541C
:106B10004854203F202020202020202000266BF2F7
:106B20006A0300530300534C2041494C202020208D
:106B300020202020202000466B0C6B0140540300D5
:106B400000FF007E0000534C20454C4520202020B3
:106B500020202020202000666B266B014056030079
:106B600000FF007E0000534C20525544202020207E
:106B700020202020202000866B466B014058030017
:106B800000FF007E0000534C205448542020202059
:106B900020202020202000A66B666B01405A0300B5
:106BA00000FF007E0000534C2041494C203F202034
:106BB00020202020202000C06B866B03005503009E
:106BC000534C20454C45203F2020202020202020D1
:106BD00000DA6BA66B0300570300534C2052554458
:106BE000203F202020202020202000F46BC06B03B9
:106BF00000590300534C20544854203F20202020AB
:106C000020202020000E6CDA6B03005B0300455847
:106C10004954202020202020202020202020003E19
:106C20006AF46B0300CD00002020202041696C65D0
:106C3000726F6E202020202000486C426D09865C17
:106C40006D0000145AC2590020202020456C657642
:106C500061746F722020202000686C286C09865CAB
:106C60006D0000425AEC590020202020205275640B
:106C7000646572202020202000886C486C09865CA6
:106C80006D0000505A005A00202020205468726F76
:106C900074746C652020202000A86C686C098652F2
:106CA0006E0000B85A5E5A00202020202020434861
:106CB000352020202020202000C86C886C098644C4
:106CC0006F00006A5B1A5B002020202020204348D0
:106CD000362020202020202000E86CA86C09864463
:106CE0006F0000905B425B00202020202020434862
:106CF000372020202020202000086DC86C09864401
:106D00006F00009E5B565B0020202020202043481F
:106D1000382020202020202000286DE86C09869A49
:106D20006F0000CE5BAC5B002020202053756220FA
:106D30005472696D7320202000426D086D09800E29
:106D40007000455849542020202020202020202059
:106D5000202000286C286D0300CD000052542F44E1
:106D6000574E20202020202020202020007A6D381F
:106D70006E0202D0000000F45B0043656E74657221
:106D80002020202020202020202000986D5C6D02F3
:106D900002D2000000F45B004C542F5550202020FC
:106DA000202020202020202000B66D7A6D0202D401
:106DB000000000F45B004475616C20526174652032
:106DC00020202020202000D06D986D0100D60000EA
:106DD0005472696D20202020202020202020202097
:106DE00000EA6DB66D0100D70000415420525354A3
:106DF0002020202020202020202000046ED06D03A1
:106E000000DB00004578706F2048492020202020BA
:106E100020202020001E6EEA6D0100D90000457878
:106E2000706F204C4F572020202020202020003839
:106E30006E046E0100DA00004558495420202020DD
:106E40002020202020202020005C6D1E6E0300CD1D
:106E50000000486967682020202020202020202072
:106E6000202000706EE26E020332034000F45B00EB
:106E70004C6F772020202020202020202020202040
:106E8000008E6E526E020334034000F45B005472B5
:106E9000696D20202020202020202020202000A8F4
:106EA0006E706E01003603005472696D204D6F6480
:106EB000652020202020202000C46E8E6E0000FC63
:106EC0006E370300507265736574202020202020E7
:106ED0002020202000E26EA86E020338034000F458
:106EE0005B004558495420202020202020202020CD
:106EF000202000526EC46E0300CD00005472696DF4
:106F0000204D6F6465204E4F524D414C00146F2C44
:106F10006F0000005472696D204D6F646520202061
:106F2000204C4F57002C6FFC6E0100005472696DAD
:106F3000204D6F64652020204849474800FC6E14AE
:106F40006F020000486967682F55702020202020BC
:106F50002020202000626F806F0202D0000000F429
:106F60005B004C6F772F44574E202020202020209C
:106F7000202000806F446F0202D2000000F45B000A
:106F80004558495420202020202020202020202047
:106F900000446F626F0300CD0000412020202020BC
:106FA0002020202020202020202000B86FF46F0215
:106FB00003D0004800F45B00422020202020202045
:106FC000202020202020202000D66F9A6F0203D29C
:106FD000004800F45B0043202020202020202020B7
:106FE00020202020202000F46FB86F0203D4004836
:106FF00000F45B0045584954202020202020202008
:1070000020202020009A6FD66F0300CD0000416938
:107010006C65726F6E202020202020202020002C04
:1070200070FE70010208040000E84A00456C6576B5
:1070300061746F722020202020202020004A700ED2
:1070400070010209040000E84A0052756464657228
:10705000202020202020202020200068702C70017B
:10706000020A040000E84A005468726F74746C6588
:1070700020202020202020200086704A7001020B52
:10708000040000E84A00434835202020202020202A
:1070900020202020202000A470687001020C040031
:1070A00000E84A00434836202020202020202020CD
:1070B0002020202000C270867001020D040000E82C
:1070C0004A00434837202020202020202020202054
:1070D000202000E070A47001020E040000E84A00C5
:1070E000434838202020202020202020202020203D
:1070F00000FE70C27001020F040000E84A004578EB
:107100006974202020202020202020202020000E14
:1071100070E0700300CD00004E6F6E650024717842
:10712000710000002041494C0030711871010000CD
:1071300020454C45003C712471020000205255440A
:107140000048713071030000205448540054713CD1
:10715000710400002043483500607148710500004B
:1071600020434836006C71547106000020434837B4
:107170000078716071070000204348380018716C76
:1071800071080000202020204D49584552203141EF
:107190002020202000A4713C740986A4745C035450
:1071A0005C065C00202020204D4958455220314289
:1071B0002020202000C47184710986A474610354C6
:1071C0005C065C00202020204D4958455220314368
:1071D0002020202000E471A4710986A47466035461
:1071E0005C065C00202020204D4958455220314447
:1071F00020202020000472C4710986A4746B0354FB
:107200005C065C00202020204D4958455220324128
:1072100020202020002472E4710986A47470035495
:107220005C065C00202020204D4958455220324207
:107230002020202000447204720986A4747503542F
:107240005C065C00202020204D49584552203243E6
:107250002020202000647224720986A4747A0354CA
:107260005C065C00202020204D49584552203244C5
:107270002020202000847244720986A4747F035465
:107280005C065C00202020204D49584552203341A7
:107290002020202000A47264720986A47484035400
:1072A0005C065C00202020204D4958455220334286
:1072B0002020202000C47284720986A4748903549B
:1072C0005C065C00202020204D4958455220334365
:1072D0002020202000E472A4720986A4748E035436
:1072E0005C065C00202020204D4958455220334444
:1072F00020202020000473C4720986A474930354D0
:107300005C065C0020202041494C20746F205255BF
:1073100044202020002473E472098656749303A04D
:107320005C965C0020202052554420746F20414917
:107330004C2020200044730473098656749303B4D0
:107340005CAA5C0020202052554420746F20454CDC
:10735000452020200064732473098656749303C863
:107360005CBE5C0020202054485420746F20454CA3
:10737000452020200080734473018816043A690078
:107380002020202020565441494C2020202020201D
:10739000009C7364730388980350680020202020A9
:1073A00020454C45564F4E202020202000B87380A9
:1073B0007303889903506800202020204455414CD5
:1073C0002041494C2020202000D2739C730980AAC0
:1073D0007500202020204455414C20454C4520205C
:1073E000202000EC73B8730980467600202020200E
:1073F00054485420484F4C4420202020000674D28A
:107400007309809476002020202049444C45202098
:10741000555020202020002074EC730980E2760073
:1074200020204D6978657220206F7264657220207B
:10743000003C7406740388A403CE68004558495480
:1074400020202020202020202020202000847120A7
:10745000740300CD0000506F73206761696E2020B7
:107460002020202020200070748A740100DF00009A
:107470004E6567206761696E202020202020202033
:10748000008A7456740100E00000455849542020D9
:1074900020202020202020202020005674707403FB
:1074A00000CD000046726F6D20202020202020207B
:1074B0002020202000BE7490750400DC0000546180
:1074C000626C65202020202020202020202000DA4F
:1074D00074A47400004A77E40000546F2020202038
:1074E0002020202020202020202000F474BE7404BE
:1074F00000DD00005265706C616365202020202053
:1075000020202020000E75DA740300E300005A509A
:107510002020202020202020202020202020002883
:1075200075F4740100DE0000506F73206761696EAE
:1075300020202020202020200042750E750100DF31
:107540000000506F7320496E6420202020202020EE
:107550002020005C7528750400E100004E6567205E
:107560006761696E2020202020202020007675424F
:10757000750100E000004E656720496E6420202000
:107580002020202020200090755C750400E200007F
:107590004558495420202020202020202020202031
:1075A00000A47476750300CD0000456E61626C65C1
:1075B0002020202020202020202000C4752C7603AD
:1075C000009A03005265762043483720202020206F
:1075D0002020202000DE75AA7503009B030044498B
:1075E000464620202020202020202020202000F897
:1075F00075C47501009C0300466C6170202020203A
:107600002020202020202020001276DE7501009D01
:10761000030043524F5720202020202020202020EC
:107620002020002C76F8750300C603004558495405
:1076300020202020202020202020202000AA751299
:10764000760300CD0000456E61626C65202020202D
:107650002020202020200060767A76030017040086
:1076600052657620434836202020202020202020EC
:10767000007A7646760300180400455849542020C5
:107680002020202020202020202000467660760325
:1076900000CD0000456E61626C6520202020202016
:1076A0002020202000AE76C87603009E0300506F95
:1076B000736974696F6E202020202020202000C86C
:1076C00076947601009F03004558495420202020DD
:1076D0002020202020202020009476AE760300CDAC
:1076E0000000456E61626C65202020202020202053
:1076F000202000FC7630770300A00300506F7369F0
:1077000074696F6E2041202020202020001677E22F
:10771000760100A10300506F736974696F6E204297
:10772000202020202020003077FC760100A20300DA
:10773000455849542020202020202020202020208F
:1077400000E27616770300CD00005461626C65207C
:107750002020202020204E6F6E650062773A78004E
:1077600000004169726372616674205461626C65E5
:107770002031007A774A77090000416972637261AB
:107780006674205461626C65203200927762770AD9
:107790000000476C6F6162616C205461626C65200F
:1077A000203100AA777A77010000476C6F6162612F
:1077B0006C205461626C6520203200C2779277029F
:1077C0000000476C6F6162616C205461626C6520DF
:1077D000203300DA77AA77030000476C6F6162619B
:1077E0006C205461626C6520203400F277C277040B
:1077F0000000476C6F6162616C205461626C6520AF
:107800002035000A78DA77050000476C6F61626105
:107810006C205461626C65202036002278F2770675
:107820000000476C6F6162616C205461626C65207E
:107830002037003A780A78070000476C6F61626170
:107840006C205461626C65202038004A77227808E9
:107850000000202020202041494C2044522020209C
:107860002020006C78407A0680AE03002020202083
:1078700020454C452044522020202020008678526C
:10788000780680AF03002020202020525544204459
:1078900052202020202000A0786C780680B00300C1
:1078A00020202020205052455345542020202020C5
:1078B00000BA7886780680B10300202020204D4948
:1078C0005845522020312020202000D478A078066E
:1078D00080B20300202020204D49584552202032FC
:1078E0002020202000EE78BA780680B30300202004
:1078F00020204D49584552202033202020200008C8
:1079000079D4780680B4030020202020202043482A
:107910003520202020202020002279EE780680B516
:107920000300202020204155544F205452494D201F
:107930002020003C7908790680B603002020202012
:107940002043483820412020202020200056792242
:10795000790680B7030020202020204348382042A9
:107960002020202020200070793C790680B8030078
:107970002020202020434838204320202020202081
:10798000008A7956790680B9030020202020534EC2
:107990004150202052202020202000A47970790618
:1079A00080BB030020202020534E415020204C203B
:1079B0002020202000BE798A790680BC0300205454
:1079C00068726F74746C652020486F6C642000D8F6
:1079D00079A4790680C2030020202049646C6520C8
:1079E000557020203120202000F279BE790680C316
:1079F000030020202049646C65205570202032202F
:107A00002020000C7AD8790680C403002020202092
:107A1000202043524F5720202020202000267AF299
:107A2000790680C50300205472696767657220502B
:107A30006F696E74732000407A0C7A09805A7A005C
:107A4000455849542020202020202020202020207C
:107A5000005278267A0300CD000041696C65726F90
:107A60006E205472696720506F7300767ACA7A016B
:107A700088C903286900456C657661746F7220546B
:107A8000726720506F7300927A5A7A0188CA03286D
:107A900069005275646465722020547269672050D1
:107AA0006F7300AE7A767A0188CB03286900546838
:107AB000726F74746C652054726720506F7300CAC3
:107AC0007A927A0188CC03286900455849542020CD
:107AD00020202020202020202020005A7AAE7A0367
:107AE00000CD0000202020202020204F4E202020EC
:107AF0002020202000FC7A447E100000202020203E
:107B00002020204F464620202020202000147BE407
:107B10007A200000535741202020202020202020C0
:107B200020204F4E002C7BFC7A0000005357412050
:107B30002020202020202020204F464600447B1477
:107B40007B8000005357422020202020202020202E
:107B500020204F4E005C7B2C7B01000053574220BD
:107B60002020202020202020204F464600747B44E7
:107B70007B810000535743202020202020202020FC
:107B800020204F4E008C7B5C7B020000535743202B
:107B90002020202020202020204F464600A47B7457
:107BA0007B8200005357442020202020202020509A
:107BB0005245535300BC7B8C7B83000053574420B9
:107BC000202020202052454C4541534500D47BA421
:107BD0007B03000053574520202020202020202018
:107BE00020204F4E00EC7BBC7B0400005357452007
:107BF0002020202020202020204F464600047CD436
:107C00007B84000053574620202020202020202065
:107C100020204F4E001C7CEC7B0500005357462073
:107C20002020202020202020204F464600347C04A5
:107C30007C85000053574720202020202020202032
:107C400020204F4E004C7C1C7C06000053574720E0
:107C50002020202020202020204F464600647C3415
:107C60007C86000053574820202020202020202000
:107C700020204F4E007C7C4C7C070000535748204E
:107C80002020202020202020204F464600947C6485
:107C90007C8700005357492020202020202020509E
:107CA0005245535300AC7C7C7C89000053574920DB
:107CB000202020202052454C4541534500C47C944F
:107CC0007C09000053574A2020202020202020201B
:107CD0002020204100DC7CAC7C8B000053574A20E4
:107CE00020202020202020202020204200F47CC4BE
:107CF0007C4B000053574A202020202020202020A9
:107D000020202043000C7DDC7C8C000053574B204E
:107D1000202020202020202020204F4E00247DF4F1
:107D20007C0D000053574B202020202020202020B5
:107D3000204F4646003C7D0C7D8D000053574C2063
:107D400020202020202020505245535300547D24D1
:107D50007D8E000053574C20202020202052454C7F
:107D600045415345006C7D3C7D0E000053574D202E
:107D700020202020202020505245535300847D5441
:107D80007D8F000053574D20202020202052454C4D
:107D900045415345009C7D6C7D0F000041696C6539
:107DA000726F6E202020202020204F4E00B47D8452
:107DB0007D30000041696C65726F6E2020202020AC
:107DC000204F464600CC7D9C7DB00000456C65761A
:107DD00061746F722020202020204F4E00E47DB47B
:107DE0007D310000456C657661746F722020202023
:107DF000204F464600FC7DCC7DB100005275646486
:107E0000657220202020202020204F4E00147EE488
:107E10007D3200005275646465722020202020208D
:107E2000204F4646002C7EFC7DB200005468726FE5
:107E300074746C652020202020204F4E00447E1456
:107E40007E3300005468726F74746C6520202020AB
:107E5000204F464600E47A2C7EB3000020202041CB
:107E600075746F20205472696D20202000767E800A
:107E70007F09801081005265736574204175746FAD
:107E8000205472696D7300947E5C7E038CDB00620B
:107E900068D25C002020205472696D20205A6572DF
:107EA0006F20202000B27E767E038CDB007468E2B7
:107EB0005C00436C656172205472696D205A657272
:107EC0006F7300D07E947E038CDB008668325D0089
:107ED00020416C74202020416972637261667420B5
:107EE00000EA7EB27E09809A7F0020436F7079207D
:107EF00020416972637261667420000A7FD07E053A
:107F00008EDD00AA68565D485D0020205365742010
:107F100044656661756C7473202000287FEA7E03D7
:107F20008CDB006268445E004E756D202070726FBD
:107F30007020626C6164657300487F0A7F05C8A584
:107F400003BC6801000500005265747261637473BC
:107F5000205761726E696E6700647F287F0388A670
:107F600003506800204155584F555420436F6E749C
:107F7000726F6C2000807F487F0080CC81BA020045
:107F80004558495420202020202020202020202037
:107F9000005C7E647F0300CD000020416C742023D0
:107FA0003120202020202020202000BA7FF68005CC
:107FB00040CF030000000060000020416C742020CE
:107FC0002331205377697463682000D47F9A7F0639
:107FD00080CE030020416C742023322020202020FA
:107FE0002020202000F47FBA7F0540D1030000004C
:107FF0000060000020416C742020233220537769F8
:1080000074636820000E80D47F0680D00300204176
:108010006C74202333202020202020202020002EBC
:1080200080F47F0540D30300000000600000204181
:108030006C742020233320537769746368200048D0
:10804000800E800680D2030020416C7420233420EF
:1080500020202020202020200068802E800540D570
:10806000030000000060000020416C7420202334D5
:10807000205377697463682000828048800680D42A
:10808000030020416C742023352020202020202054
:10809000202000A28068800540D703000000006017
:1080A000000020416C7420202335205377697463CD
:1080B000682000BC8082800680D6030020416C745A
:1080C00020233620202020202020202000DC80A219
:1080D000800540D9030000000060000020416C745E
:1080E00020202336205377697463682000F680BC13
:1080F000800680D8030045584954202020202020A5
:10810000202020202020009A7FDC800300CD00006A
:108110004154206D6F6465202020202020202020E5
:10812000002C817E8100009881B6020041542073AA
:1081300074657020202020202020202000468110FF
:108140008105009E02004154207469636B732020F6
:108150002020202020200060812C8105009F02002B
:10816000746F20545A2020202020202020202020FE
:10817000007E8146810304DB000000825D004558DB
:1081800049542020202020202020202020200010C2
:108190008160810300CD00004154206D6F64652033
:1081A0002020202020496E6300B281B2810000B6F9
:1081B00002004154206D6F6465204F6E6520536846
:1081C0006F7400988198810100B602002020202061
:1081D00020202043483120202020202000E4818CD2
:1081E000820100002020202020202043483220202F
:1081F0002020202000FC81CC8103000020202020B2
:10820000202020434833202020202020001482E416
:1082100081050000202020202020204348342020F9
:1082200020202020002C82FC81070000202020201C
:108230002020204348352020202020200044821484
:1082400082090000202020202020204348362020C2
:1082500020202020005C822C820B00002020202087
:1082600020202043483720202020202000748244F2
:10827000820D00002020202020202043483820208C
:1082800020202020008C825C820F000020202020F3
:1082900020202050504D20202020202000CC817410
:1082A0008280000020202042756464792020426F83
:1082B0007820202000BE82D8820980F2820020200F
:1082C0002020205461626C6573202020202000D87B
:1082D00082A48209808C83004558495420202020A4
:1082E000202020202020202000A482BE820300CD58
:1082F00000004D6173746572203F202020202020F3
:108300002020000C8342830300A1020020204D6145
:108310007374657220204D6F64652020002883F2FD
:108320008200005C83B7020053747564656E74202C
:108330003F202020202020200042830C830300A027
:1083400002004558495420202020202020202020B1
:10835000202000F28228830300CD00004D204D6FC5
:1083600064653D4D6963726F537461720074837408
:10837000830000004D204D6F64653D467574616259
:1083800061202020005C835C8301000041697263EE
:1083900072616674205461626C65203100AC83CCDC
:1083A000840986E684DA03505E565E004169726392
:1083B00072616674205461626C65203200CC838CDB
:1083C000830986E684E503505E565E00476C6F6263
:1083D000616C20205461626C6520203100EC83AC1C
:1083E000830986E6844602505E565E00476C6F62E3
:1083F000616C20205461626C65202032000C84CCBA
:10840000830986E6845102505E565E00476C6F62B7
:10841000616C20205461626C65202033002C84EC58
:10842000830986E6845C02505E565E00476C6F628C
:10843000616C20205461626C65202034004C840CF7
:10844000840986E6846702505E565E00476C6F6260
:10845000616C20205461626C65202035006C842C96
:10846000840986E6847202505E565E00476C6F6235
:10847000616C20205461626C65202036008C844C35
:10848000840986E6847D02505E565E00476C6F620A
:10849000616C20205461626C6520203700AC846CD4
:1084A000840986E6848802505E565E00476C6F62DF
:1084B000616C20205461626C6520203800CC848C73
:1084C000840986E6849302505E565E0045584954FE
:1084D000202020202020202020202020008C83AC61
:1084E000840300CD0000504F532030202020202056
:1084F00020202020202000008504860100D00000DC
:10850000504F5320312020202020202020202020C8
:10851000001A85E6840100D10000504F532032201C
:1085200020202020202020202020003485008501CC
:1085300000D20000504F5320332020202020202044
:1085400020202020004E851A850100D30000504FC6
:1085500053203420202020202020202020200068AC
:108560008534850100D40000504F53203520202051
:1085700020202020202020200082854E850100D54B
:108580000000504F53203620202020202020202083
:108590002020009C8568850100D60000504F5320A4
:1085A00037202020202020202020202000B6858277
:1085B000850100D70000504F532038202020202074
:1085C00020202020202000D0859C850100D800009C
:1085D000504F5320392020202020202020202020F0
:1085E00000EA85B6850100D90000504F5320313094
:1085F00020202020202020202020000486D085015B
:1086000000DA000045584954202020202020202056
:108610002020202000E684EA850300CD00002054BD
:108620005820566F6C7420204D6574657220003A96
:1086300086BC870788A45EE06800545820416C61BE
:10864000726D20566F6C74616765005A861E8608CD
:10865000C8B902E0680000FF00005265736574202D
:10866000426174742054696D65720078863A86039D
:108670008CDB006268DC5E0020525820566F6C7400
:1086800020204D65746572200094865A860788C044
:108690005EE06800536572766F20204D696E205051
:1086A000756C736500B486788602C8AE02F268E81D
:1086B00003881300536572766F20204D6178205037
:1086C000756C736500D486948602C8B002F268E8BF
:1086D000038813004E756D62657220204368616ED9
:1086E0006E656C7300F886B48605CEA20204690438
:1086F000000900885E905E0020202053796E632080
:108700007769647468202020001887D48602C8A383
:1087100002F268C800DC05002020536869667420F6
:10872000496E766572742020003487F8860388CD00
:10873000031669002020466F726D617420466C61DB
:1087400073682020004E8718870780EE5E00202087
:108750002020436F6E66696775726520202000686F
:10876000873487098036880020204A6F79537469DE
:10877000636B2043616C20200082874E870980F262
:108780008A0020202020202020464D532020202019
:10879000202000A0876887038CE9005068985E005D
:1087A000204672657175656E63792042616E642042
:1087B00000BC8782870080D687D102004558495483
:1087C000202020202020202020202020001E86A0E5
:1087D000870300CD000020202020204E6F20205253
:1087E00046202020202000EE871E88000000202048
:1087F000202020353020204D487A202020200006DF
:1088000088D6870100002020202020353320204DED
:10881000487A20202020001E88EE870200002020B9
:10882000202020373220204D487A2020202000D6DA
:108830008706880300004F75747075742063686143
:108840006E6E656C203100528886890001A0890017
:1088500004004F7574707574206368616E6E656C8A
:108860002032006E8836880001A0890104004F750F
:1088700074707574206368616E6E656C2033008A55
:108880008852880001A0890204004F7574707574C5
:10889000206368616E6E656C203400A6886E880067
:1088A00001A0890304004F757470757420636861BA
:1088B0006E6E656C203500C2888A880001A089042C
:1088C00004004F7574707574206368616E6E656C1A
:1088D000203600DE88A6880001A0890504004F75B7
:1088E00074707574206368616E6E656C203700FA71
:1088F00088C2880001A0890604004F7574707574E1
:10890000206368616E6E656C2038001689DE880011
:1089100001A08907040053656C6563742041696C8C
:1089200020205472696D003289FA880001708AB281
:10893000020053656C65637420456C652020547299
:10894000696D004E8916890001708AB30200536573
:108950006C6563742052756420205472696D006ADE
:108960008932890001708AB4020053656C656374B2
:108970002054687420205472696D0086894E8900E5
:1089800001708AB50200455849542020202020203B
:108990002020202020200036886A890300CD000096
:1089A0002020202041696C65726F6E2020202020DD
:1089B00000BA89568A0100DC000020202020456C86
:1089C000657661746F722020202000D489A089020E
:1089D00000DC000020202020205275646465722095
:1089E0002020202000EE89BA890300DC000020202E
:1089F00020205468726F74746C6520202020000859
:108A00008AD4890400DC000020202020202020437C
:108A1000483520202020202000228AEE890500DC15
:108A20000000202020202020204348362020202025
:108A30002020003C8A088A0600DC0000202020203C
:108A400020202043483720202020202000568A2242
:108A50008A0700DC00002020202020202043483806
:108A600020202020202000A0893C8A0800DC000073
:108A7000202020204E6F20205472696D202020205D
:108A8000008A8AD88A0000DC0000202020202054A0
:108A900072696D2031202020202000A48A708A0174
:108AA00000DC000020202020205472696D2032203C
:108AB0002020202000BE8A8A8A0200DC00002020BC
:108AC0002020205472696D2033202020202000D8DF
:108AD0008AA48A0300DC0000202020202054726930
:108AE0006D2034202020202000708ABE8A0400DC03
:108AF00000002020202041696C65726F6E202020CC
:108B00002020000E8B0A8C0780AE60150400202008
:108B10002020456C657661746F7220202020002A29
:108B20008BF28A0780AE601B050020202020527542
:108B30006464657220202020202000468B0E8B0765
:108B400080AE60210600202020205468726F74746B
:108B50006C652020202000628B2A8B0780E05F2735
:108B600007002020202020204348362020202020DD
:108B70002020007E8B468B0780F45E3B0000202087
:108B80002020202043483720202020202020009A29
:108B90008B628B0780F45E3F0100202041696C6589
:108BA000726F6E207472696D202000B68B7E8B0709
:108BB00080F45E2B080020456C657661746F72202E
:108BC000207472696D2000D28B9A8B0780F45E2F1F
:108BD0000900202052756464657220207472696DEA
:108BE000202000EE8BB68B0780F45E330A00205401
:108BF00068726F74746C6520207472696D20000A4D
:108C00008CD28B0780F45E370B0045786974202086
:108C10002020202020202020202000F28AEE8B031C
:108C200000CD00002020202043656E746572202056
:108C300020202020000020202052696768742F44E3
:108C40006F776E2020200000202020204C65667465
:108C50002F55702020202020000001000F00D2009E
:108C600000000300D20000001E00D2000080121B92
:108C700001660379013C012E03AE01130126039521
:108C80000162017300860412018B040701C8040508
:108C9000012A042901320237023B022F0200000898
:108CA0000001040910192431405164001324334099
:108CB0004B545B60636400010203060C15223349C8
:108CC00064001B31424F585E61626364000A141EE7
:108CD00028323C46505A640014283C5064503C28CA
:108CE000140000050A0F14192837465564000F1E9A
:108CF0002D3C4B50555A5F640A0A0000109001FF4A
:108D000000A5E7C009F30000DC059411010203048B
:108D10000000FF5801000102830405060708090A44
:108D20000B8C8D0E0F000000000000000000000002
:108D30000000000000000000000000000000000033
:108D40000000000000000000000000000000000023
:108D5000000000000000000000004D4F44454C2082
:108D600030312020202020202020000001B80B00DE
:108D7000013C190000000001B80B00013C19000083
:108D8000000001B80B00013C1900000000FEA00F1C
:108D90001901D0070001B80B0001B80B0001B80B96
:108DA0000001B80B000132FF320032003200CEFF6A
:108DB000CE00CE00CE0000000014140000000A0A0D
:108DC0000000000A0A0000000A0A0000F4010A007C
:108DD00000000A0A0000000A0A0000000A0A000057
:108DE000000A0A0000000A0A0000000A0A00000047
:108DF0000A0A000000000000000A00000000000253
:108E000000000000000000FF0001028304050607C7
:108E1000898B4B8C0D8E8F0100081000074B8C0442
:108E200000200000000000FF0D00200020002000B6
:108E30002000200000010409101924314051640071
:108E4000132433404B545B60636400000000000057
:108E500000000000000000000000020103040506FD
:108E600007080000000000000000000000000000F3
:108E700000000000000000000000000000000000F2
:108E800000000000000000000000000000000000E2
:108E900000000000000000000000000000000000D2
:108EA00000000000000000000000000000000000C2
:108EB00000000000000000000000000000000000B2
:108EC00000000000000000000000000000000000A2
:108ED0000000000000000000000000000000000092
:108EE0000000000000000000000000000000000082
:108EF0000000000000000000000000000000000072
:108F00000000000000000000000000000000000061
:108F10000000000000000000000000000000000051
:108F20000000000000000000000000000000000041
:108F30000000000000000000000000000000000031
:108F40000000000000000000000000000000000021
:0A8F50000000000000000000000017
:00000001FF
